 AddToBootstrapClassLoaderSearch

 Timestamp is 54f83cd4 (reproducible build file hash)

 Preferred load address is 0000000180000000

 Start         Length     Name                   Class
 0001:00000000 00002ef0H .text$mn                CODE
 0001:00002ef0 00000036H .text$mn$00             CODE
 0001:00002f26 00000092H .text$x                 CODE
 0002:00000000 000001a8H .idata$5                DATA
 0002:000001a8 00000038H .00cfg                  DATA
 0002:000001e0 00000008H .CRT$XCA                DATA
 0002:000001e8 00000008H .CRT$XCZ                DATA
 0002:000001f0 00000008H .CRT$XIA                DATA
 0002:000001f8 00000008H .CRT$XIC                DATA
 0002:00000200 00000008H .CRT$XIZ                DATA
 0002:00000208 00000008H .CRT$XLA                DATA
 0002:00000210 00000008H .CRT$XLZ                DATA
 0002:00000218 00000008H .CRT$XPA                DATA
 0002:00000220 00000008H .CRT$XPZ                DATA
 0002:00000228 00000008H .CRT$XTA                DATA
 0002:00000230 00000010H .CRT$XTZ                DATA
 0002:00000238 00000000H .gehcont$y              DATA
 0002:00000238 00000000H .gfids$y                DATA
 0002:00000240 00001e40H .rdata                  DATA
 0002:00002080 00000000H .rdata$CastGuardVftablesA DATA
 0002:00002080 00000000H .rdata$CastGuardVftablesC DATA
 0002:00002080 00000028H .rdata$T                DATA
 0002:000020a8 000000a4H .rdata$voltmd           DATA
 0002:0000214c 0000032cH .rdata$zzzdbg           DATA
 0002:00002478 00000008H .rtc$IAA                DATA
 0002:00002480 00000008H .rtc$IZZ                DATA
 0002:00002488 00000008H .rtc$TAA                DATA
 0002:00002490 00000008H .rtc$TZZ                DATA
 0002:00002498 00000004H .tls                    DATA
 0002:0000249c 00000004H .tls$                   DATA
 0002:000024a0 00000008H .tls$ZZZ                DATA
 0002:000024a8 000002f8H .xdata                  DATA
 0002:000027a0 000003d4H .edata                  DATA
 0002:00002b74 00000064H .idata$2                DATA
 0002:00002bd8 00000018H .idata$3                DATA
 0002:00002bf0 000001a8H .idata$4                DATA
 0002:00002d98 00000432H .idata$6                DATA
 0003:00000000 00000c40H .data                   DATA
 0003:00000c40 0001b388H .bss                    DATA
 0004:00000000 000003ccH .pdata                  DATA

  Address         Publics by Value              Rva+Base               Lib:Object

 0000:00000000       __AbsoluteZero             0000000000000000     <absolute>
 0000:00000000       ___safe_se_handler_count   0000000000000000     <absolute>
 0000:00000000       ___safe_se_handler_table   0000000000000000     <absolute>
 0000:00000000       __arm64x_extra_rfe_table   0000000000000000     <absolute>
 0000:00000000       __arm64x_extra_rfe_table_size 0000000000000000     <absolute>
 0000:00000000       __arm64x_native_entrypoint 0000000000000000     <absolute>
 0000:00000000       __arm64x_redirection_metadata 0000000000000000     <absolute>
 0000:00000000       __arm64x_redirection_metadata_count 0000000000000000     <absolute>
 0000:00000000       __dynamic_value_reloc_table 0000000000000000     <absolute>
 0000:00000000       __enclave_config           0000000000000000     <absolute>
 0000:00000000       __guard_check_icall_a64n_fptr 0000000000000000     <absolute>
 0000:00000000       __guard_eh_cont_count      0000000000000000     <absolute>
 0000:00000000       __guard_eh_cont_table      0000000000000000     <absolute>
 0000:00000000       __guard_fids_count         0000000000000000     <absolute>
 0000:00000000       __guard_fids_table         0000000000000000     <absolute>
 0000:00000000       __guard_iat_count          0000000000000000     <absolute>
 0000:00000000       __guard_iat_table          0000000000000000     <absolute>
 0000:00000000       __guard_longjmp_count      0000000000000000     <absolute>
 0000:00000000       __guard_longjmp_table      0000000000000000     <absolute>
 0000:00000000       __hybrid_auxiliary_iat     0000000000000000     <absolute>
 0000:00000000       __hybrid_auxiliary_iat_copy 0000000000000000     <absolute>
 0000:00000000       __hybrid_code_map          0000000000000000     <absolute>
 0000:00000000       __hybrid_code_map_count    0000000000000000     <absolute>
 0000:00000000       __x64_code_ranges_to_entry_points 0000000000000000     <absolute>
 0000:00000000       __x64_code_ranges_to_entry_points_count 0000000000000000     <absolute>
 0000:00000100       __guard_flags              0000000000000100     <absolute>
 0000:00000000       __ImageBase                0000000180000000     <linker-defined>
 0001:00000000       ?NewObject@JNIEnv_@@QEAAPEAV_jobject@@PEAV_jclass@@PEAU_jmethodID@@ZZ 0000000180001000 f i libAddToBootstrapClassLoaderSearch.obj
 0001:00000028       ?SetEventNotificationMode@_jvmtiEnv@@QEAA?AW4jvmtiError@@W4jvmtiEventMode@@W4jvmtiEvent@@PEAV_jobject@@ZZ 0000000180001028 f i libAddToBootstrapClassLoaderSearch.obj
 0001:00000034       ?TranslateError@@YAPEBDW4jvmtiError@@@Z 0000000180001034 f   libAddToBootstrapClassLoaderSearch.obj
 0001:000002ec       ?nsk_jni_check_exception@@YAHPEAUJNIEnv_@@QEBDH@Z 00000001800012ec f   libAddToBootstrapClassLoaderSearch.obj
 0001:00000430       ?nsk_jni_lverify@@YAHHPEAUJNIEnv_@@HQEBDH1ZZ 0000000180001430 f   libAddToBootstrapClassLoaderSearch.obj
 0001:000004d0       Agent_Initialize           00000001800014d0 f   libAddToBootstrapClassLoaderSearch.obj
 0001:00000758       Agent_OnAttach             0000000180001758 f   libAddToBootstrapClassLoaderSearch.obj
 0001:00000758       Agent_OnLoad               0000000180001758 f   libAddToBootstrapClassLoaderSearch.obj
 0001:00000760       Java_nsk_jvmti_unit_FollowReferences_FollowRefObjects_addRefToVerify 0000000180001760 f   libAddToBootstrapClassLoaderSearch.obj
 0001:00000938       Java_nsk_jvmti_unit_FollowReferences_FollowRefObjects_getTag 0000000180001938 f   libAddToBootstrapClassLoaderSearch.obj
 0001:000009f8       Java_nsk_jvmti_unit_FollowReferences_FollowRefObjects_resetRefsToVerify 00000001800019f8 f   libAddToBootstrapClassLoaderSearch.obj
 0001:00000a00       Java_nsk_jvmti_unit_FollowReferences_FollowRefObjects_resetTags 0000000180001a00 f   libAddToBootstrapClassLoaderSearch.obj
 0001:00000a44       Java_nsk_jvmti_unit_FollowReferences_FollowRefObjects_setTag 0000000180001a44 f   libAddToBootstrapClassLoaderSearch.obj
 0001:00000c9c       Java_nsk_jvmti_unit_functions_AddToBootstrapClassLoaderSearch_JvmtiTest_GetResult 0000000180001c9c f   libAddToBootstrapClassLoaderSearch.obj
 0001:00000cd0       Java_nsk_share_jvmti_ArgumentHandler_getAgentOptionsString 0000000180001cd0 f   libAddToBootstrapClassLoaderSearch.obj
 0001:00000d80       Java_nsk_share_jvmti_DebugeeClass_checkStatus 0000000180001d80 f   libAddToBootstrapClassLoaderSearch.obj
 0001:00000e08       Java_nsk_share_jvmti_DebugeeClass_resetAgentData 0000000180001e08 f   libAddToBootstrapClassLoaderSearch.obj
 0001:00000e68       Java_nsk_share_jvmti_RedefineAgent_agentStatus 0000000180001e68 f   libAddToBootstrapClassLoaderSearch.obj
 0001:00000e74       Java_nsk_share_jvmti_RedefineAgent_isRedefined 0000000180001e74 f   libAddToBootstrapClassLoaderSearch.obj
 0001:00000e80       Java_nsk_share_jvmti_RedefineAgent_redefineAttempted 0000000180001e80 f   libAddToBootstrapClassLoaderSearch.obj
 0001:00000e8c       MA_checkStatus             0000000180001e8c f   libAddToBootstrapClassLoaderSearch.obj
 0001:00000f30       NativeMethodBind           0000000180001f30 f   libAddToBootstrapClassLoaderSearch.obj
 0001:00000fdc       __local_stdio_printf_options 0000000180001fdc f i libAddToBootstrapClassLoaderSearch.obj
 0001:000011bc       classFileLoadEvent         00000001800021bc f   libAddToBootstrapClassLoaderSearch.obj
 0001:00001214       debug_printf               0000000180002214 f   libAddToBootstrapClassLoaderSearch.obj
 0001:00001270       exitOnError                0000000180002270 f   libAddToBootstrapClassLoaderSearch.obj
 0001:00001324       fprintf                    0000000180002324 f i libAddToBootstrapClassLoaderSearch.obj
 0001:00001368       init_callbacks             0000000180002368 f   libAddToBootstrapClassLoaderSearch.obj
 0001:000013cc       nsk_jvmti_lverify          00000001800023cc f   libAddToBootstrapClassLoaderSearch.obj
 0001:000014bc       nsk_jvmti_resetAgentData   00000001800024bc f   libAddToBootstrapClassLoaderSearch.obj
 0001:0000153c       nsk_jvmti_setFailStatus    000000018000253c f   libAddToBootstrapClassLoaderSearch.obj
 0001:00001578       nsk_lcomplain              0000000180002578 f   libAddToBootstrapClassLoaderSearch.obj
 0001:00001598       nsk_ldisplay               0000000180002598 f   libAddToBootstrapClassLoaderSearch.obj
 0001:000015b8       nsk_ltrace                 00000001800025b8 f   libAddToBootstrapClassLoaderSearch.obj
 0001:000015d8       nsk_lvcomplain             00000001800025d8 f   libAddToBootstrapClassLoaderSearch.obj
 0001:00001790       nsk_lvdisplay              0000000180002790 f   libAddToBootstrapClassLoaderSearch.obj
 0001:000017dc       nsk_lverify                00000001800027dc f   libAddToBootstrapClassLoaderSearch.obj
 0001:00001838       nsk_lvtrace                0000000180002838 f   libAddToBootstrapClassLoaderSearch.obj
 0001:00001898       nsk_printf                 0000000180002898 f   libAddToBootstrapClassLoaderSearch.obj
 0001:000018c0       nsk_vprintf                00000001800028c0 f   libAddToBootstrapClassLoaderSearch.obj
 0001:00001974       printf                     0000000180002974 f i libAddToBootstrapClassLoaderSearch.obj
 0001:00001e9c       vmDeath                    0000000180002e9c f   libAddToBootstrapClassLoaderSearch.obj
 0001:00001efc       vmInit                     0000000180002efc f   libAddToBootstrapClassLoaderSearch.obj
 0001:00001f5c       vmStart                    0000000180002f5c f   libAddToBootstrapClassLoaderSearch.obj
 0001:00001fbc       __raise_securityfailure    0000000180002fbc f   MSVCRT:gs_report.obj
 0001:00001ff0       __report_gsfailure         0000000180002ff0 f   MSVCRT:gs_report.obj
 0001:00002230       __GSHandlerCheck           0000000180003230 f   MSVCRT:gshandler.obj
 0001:00002250       __GSHandlerCheckCommon     0000000180003250 f   MSVCRT:gshandler.obj
 0001:000022c0       __security_check_cookie    00000001800032c0 f   MSVCRT:amdsecgs.obj
 0001:00002600       _DllMainCRTStartup         0000000180003600 f   MSVCRT:dll_dllmain.obj
 0001:00002640       __scrt_acquire_startup_lock 0000000180003640 f   MSVCRT:utility.obj
 0001:0000267c       __scrt_dllmain_after_initialize_c 000000018000367c f   MSVCRT:utility.obj
 0001:000026b0       __scrt_dllmain_before_initialize_c 00000001800036b0 f   MSVCRT:utility.obj
 0001:000026c8       __scrt_dllmain_crt_thread_attach 00000001800036c8 f   MSVCRT:utility.obj
 0001:000026f0       __scrt_dllmain_crt_thread_detach 00000001800036f0 f   MSVCRT:utility.obj
 0001:00002708       __scrt_dllmain_exception_filter 0000000180003708 f   MSVCRT:utility.obj
 0001:00002768       __scrt_dllmain_uninitialize_c 0000000180003768 f   MSVCRT:utility.obj
 0001:00002798       __scrt_dllmain_uninitialize_critical 0000000180003798 f   MSVCRT:utility.obj
 0001:000027ac       __scrt_initialize_crt      00000001800037ac f   MSVCRT:utility.obj
 0001:000027f8       __scrt_initialize_onexit_tables 00000001800037f8 f   MSVCRT:utility.obj
 0001:00002884       __scrt_is_nonwritable_in_current_image 0000000180003884 f   MSVCRT:utility.obj
 0001:0000291c       __scrt_release_startup_lock 000000018000391c f   MSVCRT:utility.obj
 0001:00002940       __scrt_uninitialize_crt    0000000180003940 f   MSVCRT:utility.obj
 0001:0000296c       _onexit                    000000018000396c f   MSVCRT:utility.obj
 0001:000029a8       atexit                     00000001800039a8 f   MSVCRT:utility.obj
 0001:000029c0       __crt_debugger_hook        00000001800039c0 f   MSVCRT:utility_desktop.obj
 0001:000029c8       __scrt_fastfail            00000001800039c8 f   MSVCRT:utility_desktop.obj
 0001:00002b14       _guard_check_icall_nop     0000000180003b14 f i MSVCRT:guard_support.obj
 0001:00002b18       __security_init_cookie     0000000180003b18 f   MSVCRT:gs_support.obj
 0001:00002bc4       DllMain                    0000000180003bc4 f   MSVCRT:dll_dllmain_stub.obj
 0001:00002be8       ?__scrt_initialize_type_info@@YAXXZ 0000000180003be8 f   MSVCRT:tncleanup.obj
 0001:00002bf8       ?__scrt_uninitialize_type_info@@YAXXZ 0000000180003bf8 f   MSVCRT:tncleanup.obj
 0001:00002c04       __local_stdio_scanf_options 0000000180003c04 f i MSVCRT:default_local_stdio_options.obj
 0001:00002c0c       __scrt_initialize_default_local_stdio_options 0000000180003c0c f   MSVCRT:default_local_stdio_options.obj
 0001:00002c28       __scrt_get_dyn_tls_init_callback 0000000180003c28 f   MSVCRT:dyn_tls_init.obj
 0001:00002c30       _RTC_Initialize            0000000180003c30 f   MSVCRT:initsect.obj
 0001:00002c6c       _RTC_Terminate             0000000180003c6c f   MSVCRT:initsect.obj
 0001:00002ca8       __isa_available_init       0000000180003ca8 f   MSVCRT:cpu_disp.obj
 0001:00002e54       _get_startup_argv_mode     0000000180003e54 f   MSVCRT:argv_mode.obj
 0001:00002e5c       __scrt_is_ucrt_dll_in_use  0000000180003e5c f   MSVCRT:ucrt_detection.obj
 0001:00002e70       memcpy                     0000000180003e70 f   vcruntime:VCRUNTIME140.dll
 0001:00002e76       memset                     0000000180003e76 f   vcruntime:VCRUNTIME140.dll
 0001:00002e7c       strchr                     0000000180003e7c f   vcruntime:VCRUNTIME140.dll
 0001:00002e82       strstr                     0000000180003e82 f   vcruntime:VCRUNTIME140.dll
 0001:00002e88       __C_specific_handler       0000000180003e88 f   vcruntime:VCRUNTIME140.dll
 0001:00002e8e       __std_type_info_destroy_list 0000000180003e8e f   vcruntime:VCRUNTIME140.dll
 0001:00002e94       strcat                     0000000180003e94 f   ucrt:api-ms-win-crt-string-l1-1-0.dll
 0001:00002e9a       strcmp                     0000000180003e9a f   ucrt:api-ms-win-crt-string-l1-1-0.dll
 0001:00002ea0       strlen                     0000000180003ea0 f   ucrt:api-ms-win-crt-string-l1-1-0.dll
 0001:00002ea6       _initterm                  0000000180003ea6 f   ucrt:api-ms-win-crt-runtime-l1-1-0.dll
 0001:00002eac       _initterm_e                0000000180003eac f   ucrt:api-ms-win-crt-runtime-l1-1-0.dll
 0001:00002eb2       _seh_filter_dll            0000000180003eb2 f   ucrt:api-ms-win-crt-runtime-l1-1-0.dll
 0001:00002eb8       _configure_narrow_argv     0000000180003eb8 f   ucrt:api-ms-win-crt-runtime-l1-1-0.dll
 0001:00002ebe       _initialize_narrow_environment 0000000180003ebe f   ucrt:api-ms-win-crt-runtime-l1-1-0.dll
 0001:00002ec4       _initialize_onexit_table   0000000180003ec4 f   ucrt:api-ms-win-crt-runtime-l1-1-0.dll
 0001:00002eca       _register_onexit_function  0000000180003eca f   ucrt:api-ms-win-crt-runtime-l1-1-0.dll
 0001:00002ed0       _execute_onexit_table      0000000180003ed0 f   ucrt:api-ms-win-crt-runtime-l1-1-0.dll
 0001:00002ed6       _crt_atexit                0000000180003ed6 f   ucrt:api-ms-win-crt-runtime-l1-1-0.dll
 0001:00002edc       _cexit                     0000000180003edc f   ucrt:api-ms-win-crt-runtime-l1-1-0.dll
 0001:00002ee4       __acrt_initialize          0000000180003ee4 f   MSVCRT:ucrt_stubs.obj
 0001:00002ee4       __acrt_thread_attach       0000000180003ee4 f   MSVCRT:ucrt_stubs.obj
 0001:00002ee4       __acrt_thread_detach       0000000180003ee4 f   MSVCRT:ucrt_stubs.obj
 0001:00002ee4       __acrt_uninitialize        0000000180003ee4 f   MSVCRT:ucrt_stubs.obj
 0001:00002ee4       __acrt_uninitialize_critical 0000000180003ee4 f   MSVCRT:ucrt_stubs.obj
 0001:00002ee4       __scrt_stub_for_acrt_initialize 0000000180003ee4 f   MSVCRT:ucrt_stubs.obj
 0001:00002ee4       __scrt_stub_for_acrt_thread_attach 0000000180003ee4 f   MSVCRT:ucrt_stubs.obj
 0001:00002ee4       __scrt_stub_for_acrt_thread_detach 0000000180003ee4 f   MSVCRT:ucrt_stubs.obj
 0001:00002ee4       __scrt_stub_for_acrt_uninitialize 0000000180003ee4 f   MSVCRT:ucrt_stubs.obj
 0001:00002ee4       __scrt_stub_for_acrt_uninitialize_critical 0000000180003ee4 f   MSVCRT:ucrt_stubs.obj
 0001:00002ee4       __vcrt_initialize          0000000180003ee4 f   MSVCRT:ucrt_stubs.obj
 0001:00002ee4       __vcrt_thread_attach       0000000180003ee4 f   MSVCRT:ucrt_stubs.obj
 0001:00002ee4       __vcrt_thread_detach       0000000180003ee4 f   MSVCRT:ucrt_stubs.obj
 0001:00002ee4       __vcrt_uninitialize        0000000180003ee4 f   MSVCRT:ucrt_stubs.obj
 0001:00002ee4       __vcrt_uninitialize_critical 0000000180003ee4 f   MSVCRT:ucrt_stubs.obj
 0001:00002ee8       __scrt_stub_for_is_c_termination_complete 0000000180003ee8 f   MSVCRT:ucrt_stubs.obj
 0001:00002ee8       _is_c_termination_complete 0000000180003ee8 f   MSVCRT:ucrt_stubs.obj
 0001:00002f00       _guard_dispatch_icall_nop  0000000180003f00 f   MSVCRT:guard_dispatch.obj
 0001:00002f20       _guard_xfg_dispatch_icall_nop 0000000180003f20 f   MSVCRT:guard_xfg_dispatch.obj
 0002:00000000       __imp_RtlCaptureContext    0000000180004000     kernel32:KERNEL32.dll
 0002:00000008       __imp_RtlLookupFunctionEntry 0000000180004008     kernel32:KERNEL32.dll
 0002:00000010       __imp_RtlVirtualUnwind     0000000180004010     kernel32:KERNEL32.dll
 0002:00000018       __imp_UnhandledExceptionFilter 0000000180004018     kernel32:KERNEL32.dll
 0002:00000020       __imp_SetUnhandledExceptionFilter 0000000180004020     kernel32:KERNEL32.dll
 0002:00000028       __imp_GetCurrentProcess    0000000180004028     kernel32:KERNEL32.dll
 0002:00000030       __imp_TerminateProcess     0000000180004030     kernel32:KERNEL32.dll
 0002:00000038       __imp_IsProcessorFeaturePresent 0000000180004038     kernel32:KERNEL32.dll
 0002:00000040       __imp_CloseHandle          0000000180004040     kernel32:KERNEL32.dll
 0002:00000048       __imp_InitializeCriticalSectionAndSpinCount 0000000180004048     kernel32:KERNEL32.dll
 0002:00000050       __imp_DeleteCriticalSection 0000000180004050     kernel32:KERNEL32.dll
 0002:00000058       __imp_CreateEventW         0000000180004058     kernel32:KERNEL32.dll
 0002:00000060       __imp_GetModuleHandleW     0000000180004060     kernel32:KERNEL32.dll
 0002:00000068       __imp_GetProcAddress       0000000180004068     kernel32:KERNEL32.dll
 0002:00000070       __imp_IsDebuggerPresent    0000000180004070     kernel32:KERNEL32.dll
 0002:00000078       __imp_QueryPerformanceCounter 0000000180004078     kernel32:KERNEL32.dll
 0002:00000080       __imp_GetCurrentProcessId  0000000180004080     kernel32:KERNEL32.dll
 0002:00000088       __imp_GetCurrentThreadId   0000000180004088     kernel32:KERNEL32.dll
 0002:00000090       __imp_GetSystemTimeAsFileTime 0000000180004090     kernel32:KERNEL32.dll
 0002:00000098       __imp_DisableThreadLibraryCalls 0000000180004098     kernel32:KERNEL32.dll
 0002:000000a0       __imp_InitializeSListHead  00000001800040a0     kernel32:KERNEL32.dll
 0002:000000a8       \177KERNEL32_NULL_THUNK_DATA 00000001800040a8     kernel32:KERNEL32.dll
 0002:000000b0       __imp_memcpy               00000001800040b0     vcruntime:VCRUNTIME140.dll
 0002:000000b8       __imp_memset               00000001800040b8     vcruntime:VCRUNTIME140.dll
 0002:000000c0       __imp_strchr               00000001800040c0     vcruntime:VCRUNTIME140.dll
 0002:000000c8       __imp_strstr               00000001800040c8     vcruntime:VCRUNTIME140.dll
 0002:000000d0       __imp___C_specific_handler 00000001800040d0     vcruntime:VCRUNTIME140.dll
 0002:000000d8       __imp___std_type_info_destroy_list 00000001800040d8     vcruntime:VCRUNTIME140.dll
 0002:000000e0       \177VCRUNTIME140_NULL_THUNK_DATA 00000001800040e0     vcruntime:VCRUNTIME140.dll
 0002:000000e8       __imp__errno               00000001800040e8     ucrt:api-ms-win-crt-runtime-l1-1-0.dll
 0002:000000f0       __imp_exit                 00000001800040f0     ucrt:api-ms-win-crt-runtime-l1-1-0.dll
 0002:000000f8       __imp__cexit               00000001800040f8     ucrt:api-ms-win-crt-runtime-l1-1-0.dll
 0002:00000100       __imp__crt_atexit          0000000180004100     ucrt:api-ms-win-crt-runtime-l1-1-0.dll
 0002:00000108       __imp__execute_onexit_table 0000000180004108     ucrt:api-ms-win-crt-runtime-l1-1-0.dll
 0002:00000110       __imp__register_onexit_function 0000000180004110     ucrt:api-ms-win-crt-runtime-l1-1-0.dll
 0002:00000118       __imp__initialize_onexit_table 0000000180004118     ucrt:api-ms-win-crt-runtime-l1-1-0.dll
 0002:00000120       __imp__initialize_narrow_environment 0000000180004120     ucrt:api-ms-win-crt-runtime-l1-1-0.dll
 0002:00000128       __imp__configure_narrow_argv 0000000180004128     ucrt:api-ms-win-crt-runtime-l1-1-0.dll
 0002:00000130       __imp__seh_filter_dll      0000000180004130     ucrt:api-ms-win-crt-runtime-l1-1-0.dll
 0002:00000138       __imp__initterm_e          0000000180004138     ucrt:api-ms-win-crt-runtime-l1-1-0.dll
 0002:00000140       __imp__initterm            0000000180004140     ucrt:api-ms-win-crt-runtime-l1-1-0.dll
 0002:00000148       \177api-ms-win-crt-runtime-l1-1-0_NULL_THUNK_DATA 0000000180004148     ucrt:api-ms-win-crt-runtime-l1-1-0.dll
 0002:00000150       __imp___acrt_iob_func      0000000180004150     ucrt:api-ms-win-crt-stdio-l1-1-0.dll
 0002:00000158       __imp_fflush               0000000180004158     ucrt:api-ms-win-crt-stdio-l1-1-0.dll
 0002:00000160       __imp___stdio_common_vsprintf 0000000180004160     ucrt:api-ms-win-crt-stdio-l1-1-0.dll
 0002:00000168       __imp___stdio_common_vfprintf 0000000180004168     ucrt:api-ms-win-crt-stdio-l1-1-0.dll
 0002:00000170       \177api-ms-win-crt-stdio-l1-1-0_NULL_THUNK_DATA 0000000180004170     ucrt:api-ms-win-crt-stdio-l1-1-0.dll
 0002:00000178       __imp_strcat               0000000180004178     ucrt:api-ms-win-crt-string-l1-1-0.dll
 0002:00000180       __imp_strcmp               0000000180004180     ucrt:api-ms-win-crt-string-l1-1-0.dll
 0002:00000188       __imp__strdup              0000000180004188     ucrt:api-ms-win-crt-string-l1-1-0.dll
 0002:00000188       __imp_strdup               0000000180004188     ucrt:api-ms-win-crt-string-l1-1-0.dll
 0002:00000190       __imp_strlen               0000000180004190     ucrt:api-ms-win-crt-string-l1-1-0.dll
 0002:00000198       __imp_strncpy              0000000180004198     ucrt:api-ms-win-crt-string-l1-1-0.dll
 0002:000001a0       \177api-ms-win-crt-string-l1-1-0_NULL_THUNK_DATA 00000001800041a0     ucrt:api-ms-win-crt-string-l1-1-0.dll
 0002:000001a8       __guard_check_icall_fptr   00000001800041a8     MSVCRT:guard_support.obj
 0002:000001b0       __guard_xfg_check_icall_fptr 00000001800041b0     MSVCRT:guard_support.obj
 0002:000001b8       __guard_dispatch_icall_fptr 00000001800041b8     MSVCRT:guard_support.obj
 0002:000001c0       __guard_xfg_dispatch_icall_fptr 00000001800041c0     MSVCRT:guard_support.obj
 0002:000001c8       __guard_xfg_table_dispatch_icall_fptr 00000001800041c8     MSVCRT:guard_support.obj
 0002:000001d0       __castguard_check_failure_os_handled_fptr 00000001800041d0     MSVCRT:guard_support.obj
 0002:000001d8       __guard_memcpy_fptr        00000001800041d8     vcruntime:softmemtag.obj
 0002:000001e0       __xc_a                     00000001800041e0     MSVCRT:initializers.obj
 0002:000001e8       __xc_z                     00000001800041e8     MSVCRT:initializers.obj
 0002:000001f0       __xi_a                     00000001800041f0     MSVCRT:initializers.obj
 0002:00000200       __xi_z                     0000000180004200     MSVCRT:initializers.obj
 0002:00000208       __xl_a                     0000000180004208     MSVCRT:tlssup.obj
 0002:00000210       __xl_z                     0000000180004210     MSVCRT:tlssup.obj
 0002:00000218       __xp_a                     0000000180004218     MSVCRT:initializers.obj
 0002:00000220       __xp_z                     0000000180004220     MSVCRT:initializers.obj
 0002:00000228       __xt_a                     0000000180004228     MSVCRT:initializers.obj
 0002:00000230       __xt_z                     0000000180004230     MSVCRT:initializers.obj
 0002:00000240       g_refKindStr               0000000180004240     libAddToBootstrapClassLoaderSearch.obj
 0002:000003f0       ??_C@_09BPLDFGCI@unknown_0@ 00000001800043f0     libAddToBootstrapClassLoaderSearch.obj
 0002:00000400       ??_C@_0BL@FPNMECJD@JVMTI_HEAP_REFERENCE_CLASS@ 0000000180004400     libAddToBootstrapClassLoaderSearch.obj
 0002:00000420       ??_C@_0BL@FKGKKLNM@JVMTI_HEAP_REFERENCE_FIELD@ 0000000180004420     libAddToBootstrapClassLoaderSearch.obj
 0002:00000440       ??_C@_0CD@CAEHCFJF@JVMTI_HEAP_REFERENCE_ARRAY_ELEM@ 0000000180004440     libAddToBootstrapClassLoaderSearch.obj
 0002:00000468       ??_C@_0CC@DNEBMCNK@JVMTI_HEAP_REFERENCE_CLASS_LOAD@ 0000000180004468     libAddToBootstrapClassLoaderSearch.obj
 0002:00000490       ??_C@_0BN@CJMIPEBB@JVMTI_HEAP_REFERENCE_SIGNERS@ 0000000180004490     libAddToBootstrapClassLoaderSearch.obj
 0002:000004b0       ??_C@_0CH@HBOIDPEB@JVMTI_HEAP_REFERENCE_PROTECTION@ 00000001800044b0     libAddToBootstrapClassLoaderSearch.obj
 0002:000004d8       ??_C@_0BP@MDKGDGKL@JVMTI_HEAP_REFERENCE_INTERFACE@ 00000001800044d8     libAddToBootstrapClassLoaderSearch.obj
 0002:000004f8       ??_C@_0CC@JJMIHNJH@JVMTI_HEAP_REFERENCE_STATIC_FIE@ 00000001800044f8     libAddToBootstrapClassLoaderSearch.obj
 0002:00000520       ??_C@_0CD@IDHEEGID@JVMTI_HEAP_REFERENCE_CONSTANT_P@ 0000000180004520     libAddToBootstrapClassLoaderSearch.obj
 0002:00000548       ??_C@_0CA@EFFCHNG@JVMTI_HEAP_REFERENCE_SUPERCLASS@ 0000000180004548     libAddToBootstrapClassLoaderSearch.obj
 0002:00000568       ??_C@_0L@PCDFHGCJ@unknown_11@ 0000000180004568     libAddToBootstrapClassLoaderSearch.obj
 0002:00000578       ??_C@_0L@NJBICFOK@unknown_12@ 0000000180004578     libAddToBootstrapClassLoaderSearch.obj
 0002:00000588       ??_C@_0L@MAADBEKL@unknown_13@ 0000000180004588     libAddToBootstrapClassLoaderSearch.obj
 0002:00000598       ??_C@_0L@IPECICGM@unknown_14@ 0000000180004598     libAddToBootstrapClassLoaderSearch.obj
 0002:000005a8       ??_C@_0L@JGFJLDCN@unknown_15@ 00000001800045a8     libAddToBootstrapClassLoaderSearch.obj
 0002:000005b8       ??_C@_0L@LNHEOAOO@unknown_16@ 00000001800045b8     libAddToBootstrapClassLoaderSearch.obj
 0002:000005c8       ??_C@_0L@KEGPNBKP@unknown_17@ 00000001800045c8     libAddToBootstrapClassLoaderSearch.obj
 0002:000005d8       ??_C@_0L@CDPHMNGA@unknown_18@ 00000001800045d8     libAddToBootstrapClassLoaderSearch.obj
 0002:000005e8       ??_C@_0L@DKOMPMCB@unknown_19@ 00000001800045e8     libAddToBootstrapClassLoaderSearch.obj
 0002:000005f8       ??_C@_0L@OJGIPJDB@unknown_20@ 00000001800045f8     libAddToBootstrapClassLoaderSearch.obj
 0002:00000608       ??_C@_0CA@KAOFNDEM@JVMTI_HEAP_REFERENCE_JNI_GLOBAL@ 0000000180004608     libAddToBootstrapClassLoaderSearch.obj
 0002:00000628       ??_C@_0CC@HPFAJBK@JVMTI_HEAP_REFERENCE_SYSTEM_CLA@ 0000000180004628     libAddToBootstrapClassLoaderSearch.obj
 0002:00000650       ??_C@_0BN@FDEGFOHC@JVMTI_HEAP_REFERENCE_MONITOR@ 0000000180004650     libAddToBootstrapClassLoaderSearch.obj
 0002:00000670       ??_C@_0CB@HKIBCMAJ@JVMTI_HEAP_REFERENCE_STACK_LOCA@ 0000000180004670     libAddToBootstrapClassLoaderSearch.obj
 0002:00000698       ??_C@_0BP@EAACMMOE@JVMTI_HEAP_REFERENCE_JNI_LOCAL@ 0000000180004698     libAddToBootstrapClassLoaderSearch.obj
 0002:000006b8       ??_C@_0BM@IJDEOGOE@JVMTI_HEAP_REFERENCE_THREAD@ 00000001800046b8     libAddToBootstrapClassLoaderSearch.obj
 0002:000006d8       ??_C@_0BL@EDGPPKC@JVMTI_HEAP_REFERENCE_OTHER@ 00000001800046d8     libAddToBootstrapClassLoaderSearch.obj
 0002:000006f4       ??_C@_04BCJPDBDA@Code@     00000001800046f4     libAddToBootstrapClassLoaderSearch.obj
 0002:00000700       ??_C@_0BA@OCLMCFKC@LineNumberTable@ 0000000180004700     libAddToBootstrapClassLoaderSearch.obj
 0002:00000710       ??_C@_0BD@CPAEPILC@LocalVariableTable@ 0000000180004710     libAddToBootstrapClassLoaderSearch.obj
 0002:00000728       ??_C@_0BH@NMBDNHBD@LocalVariableTypeTable@ 0000000180004728     libAddToBootstrapClassLoaderSearch.obj
 0002:00000740       ??_C@_0O@HIHEEDNJ@StackMapTable@ 0000000180004740     libAddToBootstrapClassLoaderSearch.obj
 0002:00000750       ??_C@_0DO@GBNFKHHM@nsk?1jvmti?1unit?1functions?1AddToB@ 0000000180004750     libAddToBootstrapClassLoaderSearch.obj
 0002:00000790       ??_C@_0L@HCDIAMJG@?9?5?$CFs?0?5?$CFd?3?5@ 0000000180004790     libAddToBootstrapClassLoaderSearch.obj
 0002:000007a0       ??_C@_0JI@HLPECLFI@?$CD?5?4?4?4?6?$CD?5ERROR?3?5too?5many?5complai@ 00000001800047a0     libAddToBootstrapClassLoaderSearch.obj
 0002:00000840       ??_C@_0ED@JNEKCCOB@The?5following?5fake?5exception?5st@ 0000000180004840     libAddToBootstrapClassLoaderSearch.obj
 0002:00000888       ??_C@_0CN@FCNMDFBH@nsk?4share?4Fake_Exception_for_RU@ 0000000180004888     libAddToBootstrapClassLoaderSearch.obj
 0002:000008b8       ??_C@_08PGFFNAEI@?$CI?$CFs?3?$CFd?$CJ?5@ 00000001800048b8     libAddToBootstrapClassLoaderSearch.obj
 0002:000008c8       ??_C@_0DP@IENMAEGI@s?2test?2hotspot?2jtreg?2vmTestbase@ 00000001800048c8     libAddToBootstrapClassLoaderSearch.obj
 0002:00000908       ??_C@_0BL@NDJLFFJB@?7at?5nsk_lvcomplain?$CI?$CFs?3?$CFd?$CJ?6@ 0000000180004908     libAddToBootstrapClassLoaderSearch.obj
 0002:00000928       ??_C@_0BC@JOOKAFKF@?$CD?5ERROR?3?5?$CFs?0?5?$CFd?3?5@ 0000000180004928     libAddToBootstrapClassLoaderSearch.obj
 0002:00000940       ??_C@_09KJEAHMEH@?$CD?5ERROR?3?5@ 0000000180004940     libAddToBootstrapClassLoaderSearch.obj
 0002:0000094c       ??_C@_02GPIOPFAK@?$DO?$DO@ 000000018000494c     libAddToBootstrapClassLoaderSearch.obj
 0002:00000950       ??_C@_02FODMEDOG@?$DM?$DM@ 0000000180004950     libAddToBootstrapClassLoaderSearch.obj
 0002:00000954       ??_C@_02DJGKEECL@?4?4@     0000000180004954     libAddToBootstrapClassLoaderSearch.obj
 0002:00000958       ??_C@_0O@CJPGJOAF@?9?5?$CFs?0?5?$CFd?3?5?$CFs?5@ 0000000180004958     libAddToBootstrapClassLoaderSearch.obj
 0002:00000968       ??_C@_0CB@IAKPDOIC@?$CD?5?5?5verified?5assertion?5is?5FALSE@ 0000000180004968     libAddToBootstrapClassLoaderSearch.obj
 0002:00000990       ??_C@_0CO@LGONDEPD@stdout?3?5fflush?5failed?5?9?5err?$DN?$CFd?5@ 0000000180004990     libAddToBootstrapClassLoaderSearch.obj
 0002:000009c0       ??_C@_0CO@KBGKJPBD@stderr?3?5fflush?5failed?5?9?5err?$DN?$CFd?5@ 00000001800049c0     libAddToBootstrapClassLoaderSearch.obj
 0002:000009f0       ??_C@_0BB@JCNMKLLK@JVMTI_ERROR_NONE@ 00000001800049f0     libAddToBootstrapClassLoaderSearch.obj
 0002:00000a08       ??_C@_0BL@LDIMKLPH@JVMTI_ERROR_INVALID_THREAD@ 0000000180004a08     libAddToBootstrapClassLoaderSearch.obj
 0002:00000a28       ??_C@_0CB@PJFPAIKJ@JVMTI_ERROR_INVALID_THREAD_GROU@ 0000000180004a28     libAddToBootstrapClassLoaderSearch.obj
 0002:00000a50       ??_C@_0BN@LLMKHMNF@JVMTI_ERROR_INVALID_PRIORITY@ 0000000180004a50     libAddToBootstrapClassLoaderSearch.obj
 0002:00000a70       ??_C@_0CB@MBOFKAGB@JVMTI_ERROR_THREAD_NOT_SUSPENDE@ 0000000180004a70     libAddToBootstrapClassLoaderSearch.obj
 0002:00000a98       ??_C@_0BN@FABOLPBI@JVMTI_ERROR_THREAD_SUSPENDED@ 0000000180004a98     libAddToBootstrapClassLoaderSearch.obj
 0002:00000ab8       ??_C@_0BN@FDGNOBJM@JVMTI_ERROR_THREAD_NOT_ALIVE@ 0000000180004ab8     libAddToBootstrapClassLoaderSearch.obj
 0002:00000ad8       ??_C@_0BL@GOBIFKNJ@JVMTI_ERROR_INVALID_OBJECT@ 0000000180004ad8     libAddToBootstrapClassLoaderSearch.obj
 0002:00000af8       ??_C@_0BK@FCMAJPPC@JVMTI_ERROR_INVALID_CLASS@ 0000000180004af8     libAddToBootstrapClassLoaderSearch.obj
 0002:00000b18       ??_C@_0BP@IKLLBKEB@JVMTI_ERROR_CLASS_NOT_PREPARED@ 0000000180004b18     libAddToBootstrapClassLoaderSearch.obj
 0002:00000b38       ??_C@_0BN@KLPPLKG@JVMTI_ERROR_INVALID_METHODID@ 0000000180004b38     libAddToBootstrapClassLoaderSearch.obj
 0002:00000b58       ??_C@_0BN@BCEKOKND@JVMTI_ERROR_INVALID_LOCATION@ 0000000180004b58     libAddToBootstrapClassLoaderSearch.obj
 0002:00000b78       ??_C@_0BM@DFDGPME@JVMTI_ERROR_INVALID_FIELDID@ 0000000180004b78     libAddToBootstrapClassLoaderSearch.obj
 0002:00000b98       ??_C@_0BL@NELIEPEC@JVMTI_ERROR_NO_MORE_FRAMES@ 0000000180004b98     libAddToBootstrapClassLoaderSearch.obj
 0002:00000bb8       ??_C@_0BJ@BDBECFDM@JVMTI_ERROR_OPAQUE_FRAME@ 0000000180004bb8     libAddToBootstrapClassLoaderSearch.obj
 0002:00000bd8       ??_C@_0BK@MIIFNLOB@JVMTI_ERROR_TYPE_MISMATCH@ 0000000180004bd8     libAddToBootstrapClassLoaderSearch.obj
 0002:00000bf8       ??_C@_0BJ@HPCAOILC@JVMTI_ERROR_INVALID_SLOT@ 0000000180004bf8     libAddToBootstrapClassLoaderSearch.obj
 0002:00000c18       ??_C@_0BG@CHILOPNI@JVMTI_ERROR_DUPLICATE@ 0000000180004c18     libAddToBootstrapClassLoaderSearch.obj
 0002:00000c30       ??_C@_0BG@DIEMLHKM@JVMTI_ERROR_NOT_FOUND@ 0000000180004c30     libAddToBootstrapClassLoaderSearch.obj
 0002:00000c48       ??_C@_0BM@NHMCKHOB@JVMTI_ERROR_INVALID_MONITOR@ 0000000180004c48     libAddToBootstrapClassLoaderSearch.obj
 0002:00000c68       ??_C@_0BO@PPEDAJGL@JVMTI_ERROR_NOT_MONITOR_OWNER@ 0000000180004c68     libAddToBootstrapClassLoaderSearch.obj
 0002:00000c88       ??_C@_0BG@FCAIPEID@JVMTI_ERROR_INTERRUPT@ 0000000180004c88     libAddToBootstrapClassLoaderSearch.obj
 0002:00000ca0       ??_C@_0CB@EGDBNKOI@JVMTI_ERROR_INVALID_CLASS_FORMA@ 0000000180004ca0     libAddToBootstrapClassLoaderSearch.obj
 0002:00000cc8       ??_C@_0CG@DGKOGIAL@JVMTI_ERROR_CIRCULAR_CLASS_DEFI@ 0000000180004cc8     libAddToBootstrapClassLoaderSearch.obj
 0002:00000cf0       ??_C@_0BP@ICEALPKC@JVMTI_ERROR_FAILS_VERIFICATION@ 0000000180004cf0     libAddToBootstrapClassLoaderSearch.obj
 0002:00000d10       ??_C@_0DC@JDACLMIO@JVMTI_ERROR_UNSUPPORTED_REDEFIN@ 0000000180004d10     libAddToBootstrapClassLoaderSearch.obj
 0002:00000d48       ??_C@_0DE@GKDKNOMJ@JVMTI_ERROR_UNSUPPORTED_REDEFIN@ 0000000180004d48     libAddToBootstrapClassLoaderSearch.obj
 0002:00000d80       ??_C@_0BO@LAFKIOG@JVMTI_ERROR_INVALID_TYPESTATE@ 0000000180004d80     libAddToBootstrapClassLoaderSearch.obj
 0002:00000da0       ??_C@_0DH@INDGCLLB@JVMTI_ERROR_UNSUPPORTED_REDEFIN@ 0000000180004da0     libAddToBootstrapClassLoaderSearch.obj
 0002:00000dd8       ??_C@_0DE@NHEOMMGI@JVMTI_ERROR_UNSUPPORTED_REDEFIN@ 0000000180004dd8     libAddToBootstrapClassLoaderSearch.obj
 0002:00000e10       ??_C@_0CA@EKPNJOEP@JVMTI_ERROR_UNSUPPORTED_VERSION@ 0000000180004e10     libAddToBootstrapClassLoaderSearch.obj
 0002:00000e30       ??_C@_0BN@OFFMAHHL@JVMTI_ERROR_NAMES_DONT_MATCH@ 0000000180004e30     libAddToBootstrapClassLoaderSearch.obj
 0002:00000e50       ??_C@_0DN@HHBBLAKE@JVMTI_ERROR_UNSUPPORTED_REDEFIN@ 0000000180004e50     libAddToBootstrapClassLoaderSearch.obj
 0002:00000e90       ??_C@_0DO@HMBGBGNA@JVMTI_ERROR_UNSUPPORTED_REDEFIN@ 0000000180004e90     libAddToBootstrapClassLoaderSearch.obj
 0002:00000ed0       ??_C@_0BP@PBECGKHJ@JVMTI_ERROR_UNMODIFIABLE_CLASS@ 0000000180004ed0     libAddToBootstrapClassLoaderSearch.obj
 0002:00000ef0       ??_C@_0BK@CANILEHF@JVMTI_ERROR_NOT_AVAILABLE@ 0000000180004ef0     libAddToBootstrapClassLoaderSearch.obj
 0002:00000f10       ??_C@_0CE@INJKMEFK@JVMTI_ERROR_MUST_POSSESS_CAPABI@ 0000000180004f10     libAddToBootstrapClassLoaderSearch.obj
 0002:00000f38       ??_C@_0BJ@LBFPFPDM@JVMTI_ERROR_NULL_POINTER@ 0000000180004f38     libAddToBootstrapClassLoaderSearch.obj
 0002:00000f58       ??_C@_0BP@CHJPNNEM@JVMTI_ERROR_ABSENT_INFORMATION@ 0000000180004f58     libAddToBootstrapClassLoaderSearch.obj
 0002:00000f78       ??_C@_0BP@OMFMNLC@JVMTI_ERROR_INVALID_EVENT_TYPE@ 0000000180004f78     libAddToBootstrapClassLoaderSearch.obj
 0002:00000f98       ??_C@_0BN@BIBNPHHO@JVMTI_ERROR_ILLEGAL_ARGUMENT@ 0000000180004f98     libAddToBootstrapClassLoaderSearch.obj
 0002:00000fb8       ??_C@_0BK@KKNDHDCE@JVMTI_ERROR_NATIVE_METHOD@ 0000000180004fb8     libAddToBootstrapClassLoaderSearch.obj
 0002:00000fd8       ??_C@_0BK@PMKCFHAE@JVMTI_ERROR_OUT_OF_MEMORY@ 0000000180004fd8     libAddToBootstrapClassLoaderSearch.obj
 0002:00000ff8       ??_C@_0BK@NNJBDMNB@JVMTI_ERROR_ACCESS_DENIED@ 0000000180004ff8     libAddToBootstrapClassLoaderSearch.obj
 0002:00001018       ??_C@_0BI@GHECLMNC@JVMTI_ERROR_WRONG_PHASE@ 0000000180005018     libAddToBootstrapClassLoaderSearch.obj
 0002:00001030       ??_C@_0BF@OLIHJOII@JVMTI_ERROR_INTERNAL@ 0000000180005030     libAddToBootstrapClassLoaderSearch.obj
 0002:00001048       ??_C@_0BO@EOHGKJHI@JVMTI_ERROR_UNATTACHED_THREAD@ 0000000180005048     libAddToBootstrapClassLoaderSearch.obj
 0002:00001068       ??_C@_0CA@LKHFDACL@JVMTI_ERROR_INVALID_ENVIRONMENT@ 0000000180005068     libAddToBootstrapClassLoaderSearch.obj
 0002:00001088       ??_C@_0BA@MMFHLOKK@?$DMunknown?5error?$DO@ 0000000180005088     libAddToBootstrapClassLoaderSearch.obj
 0002:00001098       ??_C@_0CF@CBHOKDB@throwable?5?$DN?5jni?9?$DOExceptionOccur@ 0000000180005098     libAddToBootstrapClassLoaderSearch.obj
 0002:000010c0       ??_C@_03OFAPEBGM@?$CFs?6@  00000001800050c0     libAddToBootstrapClassLoaderSearch.obj
 0002:000010c8       ??_C@_0DM@LPIGEGNJ@s?2test?2hotspot?2jtreg?2vmTestbase@ 00000001800050c8     libAddToBootstrapClassLoaderSearch.obj
 0002:00001108       ??_C@_0CC@NFCNPEPK@Exception?5in?5JNI?5call?5?$CIcleared?$CJ@ 0000000180005108     libAddToBootstrapClassLoaderSearch.obj
 0002:00001130       ??_C@_0BJ@IBAKFIKF@jni?9?$DOExceptionDescribe?$CI?$CJ@ 0000000180005130     libAddToBootstrapClassLoaderSearch.obj
 0002:00001150       ??_C@_0BG@GGKALKMH@jni?9?$DOExceptionClear?$CI?$CJ@ 0000000180005150     libAddToBootstrapClassLoaderSearch.obj
 0002:00001168       ??_C@_0CF@JMGFGJLJ@?$CD?5?5?5verified?5JNI?5assertion?5is?5F@ 0000000180005168     libAddToBootstrapClassLoaderSearch.obj
 0002:00001190       ??_C@_0CB@MLNJNCLJ@?5?5jvmti?5error?3?5code?$DN?$CFd?0?5name?$DN?$CFs@ 0000000180005190     libAddToBootstrapClassLoaderSearch.obj
 0002:000011b8       ??_C@_0CD@OHBGDKMK@?$CD?5?5?5jvmti?5error?3?5code?$DN?$CFd?0?5name?$DN@ 00000001800051b8     libAddToBootstrapClassLoaderSearch.obj
 0002:000011e0       ??_C@_0CG@JNNCGPHB@?$CD?5?5?5error?5expected?3?5code?$DN?$CFd?0?5na@ 00000001800051e0     libAddToBootstrapClassLoaderSearch.obj
 0002:00001210       ??_C@_0EB@IMGKPCGE@?$CIstr_obj?5?$DN?5jni?9?$DONewStringUTF?$CIco@ 0000000180005210     libAddToBootstrapClassLoaderSearch.obj
 0002:00001260       ??_C@_0EA@HFOGGBCC@s?2test?2hotspot?2jtreg?2vmTestbase@ 0000000180005260     libAddToBootstrapClassLoaderSearch.obj
 0002:000012a0       ??_C@_05KKCIMGE@error@     00000001800052a0     libAddToBootstrapClassLoaderSearch.obj
 0002:000012a8       ??_C@_0CJ@JACLEAA@Test?5failed?5by?5setFailStatus?$CI?$CJ?4@ 00000001800052a8     libAddToBootstrapClassLoaderSearch.obj
 0002:000012e0       ??_C@_0EA@PNBCDMOA@s?2test?2hotspot?2jtreg?2vmTestbase@ 00000001800052e0     libAddToBootstrapClassLoaderSearch.obj
 0002:00001320       ??_C@_0DI@ILAHDLMP@?$CI?$CKagentThreadProc?$CJ?$CIjvmti_env?0?5a@ 0000000180005320     libAddToBootstrapClassLoaderSearch.obj
 0002:00001358       ??_C@_0BD@KDBALNLB@JVMTI?5agent?5thread@ 0000000180005358     libAddToBootstrapClassLoaderSearch.obj
 0002:00001370       ??_C@_0BB@NOKBFPFO@java?1lang?1Thread@ 0000000180005370     libAddToBootstrapClassLoaderSearch.obj
 0002:00001384       ??_C@_06FALKBLGB@?$DMinit?$DO@ 0000000180005384     libAddToBootstrapClassLoaderSearch.obj
 0002:00001390       ??_C@_0BG@IKDDPPGD@?$CILjava?1lang?1String?$DL?$CJV@ 0000000180005390     libAddToBootstrapClassLoaderSearch.obj
 0002:000013b0       ??_C@_0EB@IFJBFEKC@?$CIthreadClass?5?$DN?5jni_env?9?$DOFindCla@ 00000001800053b0     libAddToBootstrapClassLoaderSearch.obj
 0002:00001400       ??_C@_0GF@FGFIBKKL@?$CIthreadCtor?5?$DN?5jni_env?9?$DOGetMetho@ 0000000180005400     libAddToBootstrapClassLoaderSearch.obj
 0002:00001468       ??_C@_0DN@NCPDJLOG@?$CIthreadName?5?$DN?5jni_env?9?$DONewStrin@ 0000000180005468     libAddToBootstrapClassLoaderSearch.obj
 0002:000014b0       ??_C@_0FE@PFKODBGC@?$CIthreadObject?5?$DN?5jni_env?9?$DONewObj@ 00000001800054b0     libAddToBootstrapClassLoaderSearch.obj
 0002:00001510       ??_C@_0ED@HOBAHHJI@?$CIthreadGlobalRef?5?$DN?5jni_env?9?$DONew@ 0000000180005510     libAddToBootstrapClassLoaderSearch.obj
 0002:00001560       ??_C@_0FN@HNJJAHFC@jvmti_env?9?$DORunAgentThread?$CIagent@ 0000000180005560     libAddToBootstrapClassLoaderSearch.obj
 0002:000015c0       ??_C@_0EA@MOJDNKDF@Debuggee?5status?5sync?5aborted?5be@ 00000001800055c0     libAddToBootstrapClassLoaderSearch.obj
 0002:00001600       ??_C@_0EA@EEOEJAEN@status?5?$DN?5syncDebuggeeStatus?$CIjni@ 0000000180005600     libAddToBootstrapClassLoaderSearch.obj
 0002:00001640       ??_C@_0BL@JBCFNBMB@nsk_jvmti_resetAgentData?$CI?$CJ@ 0000000180005640     libAddToBootstrapClassLoaderSearch.obj
 0002:00001660       ??_C@_0EL@LPBEELIP@s?2test?2hotspot?2jtreg?2vmTestbase@ 0000000180005660     libAddToBootstrapClassLoaderSearch.obj
 0002:000016b0       ??_C@_0CK@JDAMFDMJ@jvmti?9?$DOSetTag?$CIo?0?5tag?$CJ?5?$DN?$DN?5JVMTI_@ 00000001800056b0     libAddToBootstrapClassLoaderSearch.obj
 0002:000016e0       ??_C@_0CC@DAMNHKNI@Can?8t?5set?5tag?5?$CFli?5for?5object?5?$CFl@ 00000001800056e0     libAddToBootstrapClassLoaderSearch.obj
 0002:00001708       ??_C@_0DL@HAJPNKEF@jvmti?9?$DOGetObjectHashCode?$CIo?0?5?$CGha@ 0000000180005708     libAddToBootstrapClassLoaderSearch.obj
 0002:00001748       ??_C@_0BL@JFPIEOBF@Can?8t?5get?5hash?5object?5?$CFlx?6@ 0000000180005748     libAddToBootstrapClassLoaderSearch.obj
 0002:00001768       ??_C@_0BG@DICPHBKN@setTag?3?5?$CF08x?5?$DM?9?5?$CF?53li@ 0000000180005768     libAddToBootstrapClassLoaderSearch.obj
 0002:00001780       ??_C@_0DH@FCEEBDMJ@?$CIs?5?$DN?5jni?9?$DOGetStringUTFChars?$CIsIn@ 0000000180005780     libAddToBootstrapClassLoaderSearch.obj
 0002:000017b8       ??_C@_0BJ@OKKGHDCN@Can?8t?5get?5string?5at?5?$CF?$CDp?6@ 00000001800057b8     libAddToBootstrapClassLoaderSearch.obj
 0002:000017d8       ??_C@_0BP@EKFLGGFJ@Can?8t?5get?5string?5at?5?$CF?$CDp?3?5null?6@ 00000001800057d8     libAddToBootstrapClassLoaderSearch.obj
 0002:000017f8       ??_C@_06ICODBHCL@?5?1?1?5?$CFs@ 00000001800057f8     libAddToBootstrapClassLoaderSearch.obj
 0002:00001800       ??_C@_0DB@KGFPLEGO@?$CIr?5?$DN?5jvmti?9?$DOGetTag?$CIo?0?5?$CGtag?$CJ?$CJ?5?$DN?$DN@ 0000000180005800     libAddToBootstrapClassLoaderSearch.obj
 0002:00001838       ??_C@_0CO@PDAGBCGJ@Can?8t?5GetTag?5for?5object?5?$CFlx?4?5Re@ 0000000180005838     libAddToBootstrapClassLoaderSearch.obj
 0002:00001868       ??_C@_0CH@HPEODOHC@TEST_BUG?3?5Max?4?5number?5of?5refs?5r@ 0000000180005868     libAddToBootstrapClassLoaderSearch.obj
 0002:00001890       ??_C@_0DI@PHFCABIM@?$CIr?5?$DN?5jvmti?9?$DOGetTag?$CIfrom?0?5?$CGtagFr@ 0000000180005890     libAddToBootstrapClassLoaderSearch.obj
 0002:000018c8       ??_C@_0DI@MDEGFNKD@TEST_BUG?3?5Can?8t?5GetTag?5for?5obje@ 00000001800058c8     libAddToBootstrapClassLoaderSearch.obj
 0002:00001900       ??_C@_0DE@MLELJAHM@?$CIr?5?$DN?5jvmti?9?$DOGetTag?$CIto?0?5?$CGtagTo?$CJ?$CJ@ 0000000180005900     libAddToBootstrapClassLoaderSearch.obj
 0002:00001938       ??_C@_0BE@MOONOKFI@VMStart?5event?5done?6@ 0000000180005938     libAddToBootstrapClassLoaderSearch.obj
 0002:00001950       ??_C@_0DJ@BHKBKNCB@VMStart?3?5AddToBootstrapClassLoa@ 0000000180005950     libAddToBootstrapClassLoaderSearch.obj
 0002:00001990       ??_C@_0BF@EAAILENF@unexpected?5error?5?$CFd?6@ 0000000180005990     libAddToBootstrapClassLoaderSearch.obj
 0002:000019a8       ??_C@_0BE@PPCKJHKJ@VMDeath?5event?5done?6@ 00000001800059a8     libAddToBootstrapClassLoaderSearch.obj
 0002:000019c0       ??_C@_0DJ@GMIIPDMD@VMDeath?3?5AddToBootstrapClassLoa@ 00000001800059c0     libAddToBootstrapClassLoaderSearch.obj
 0002:00001a00       ??_C@_0BE@EEKKELIK@VMInit?5event?5?5done?6@ 0000000180005a00     libAddToBootstrapClassLoaderSearch.obj
 0002:00001a18       ??_C@_0DI@KKGHECOA@VMInit?3?5AddToBootstrapClassLoad@ 0000000180005a18     libAddToBootstrapClassLoaderSearch.obj
 0002:00001a50       ??_C@_0BI@KCEEBAME@GetPhase?5returned?5error@ 0000000180005a50     libAddToBootstrapClassLoaderSearch.obj
 0002:00001a68       ??_C@_03PMGGPEJJ@?$CFd?6@  0000000180005a68     libAddToBootstrapClassLoaderSearch.obj
 0002:00001a70       ??_C@_0BC@PKIEGJGI@Primordial?5phase?6@ 0000000180005a70     libAddToBootstrapClassLoaderSearch.obj
 0002:00001a88       ??_C@_0DM@LNOHOIAN@Primordial?3?5AddToBootstrapClass@ 0000000180005a88     libAddToBootstrapClassLoaderSearch.obj
 0002:00001ac8       ??_C@_0DF@LIGNEPNB@Received?5class?5file?5load?5hook?5e@ 0000000180005ac8     libAddToBootstrapClassLoaderSearch.obj
 0002:00001b00       ??_C@_0BO@ENFIPLCK@Received?5class?5loader?3?50x?$CFp?5?6@ 0000000180005b00     libAddToBootstrapClassLoaderSearch.obj
 0002:00001b20       ??_C@_0BJ@DAJPLBCO@Agent_OnLoad?5event?5done?6@ 0000000180005b20     libAddToBootstrapClassLoaderSearch.obj
 0002:00001b40       ??_C@_09OPJEJKBL@printdump@ 0000000180005b40     libAddToBootstrapClassLoaderSearch.obj
 0002:00001b50       ??_C@_0CJ@KCDEKOCJ@Wrong?5result?5of?5a?5valid?5call?5to@ 0000000180005b50     libAddToBootstrapClassLoaderSearch.obj
 0002:00001b80       ??_C@_0CI@EDEMEGFA@GetPotentialCapabilities?5return@ 0000000180005b80     libAddToBootstrapClassLoaderSearch.obj
 0002:00001ba8       ??_C@_0CC@DKBFCLMH@GetAddCapabilities?5returned?5err@ 0000000180005ba8     libAddToBootstrapClassLoaderSearch.obj
 0002:00001bd0       ??_C@_0CB@NJBLABLF@SetEventCallbacks?5returned?5erro@ 0000000180005bd0     libAddToBootstrapClassLoaderSearch.obj
 0002:00001bf8       ??_C@_0DF@MIJEDHKN@SetEventNotificationMode?5for?5VM@ 0000000180005bf8     libAddToBootstrapClassLoaderSearch.obj
 0002:00001c30       ??_C@_0DE@MEFKDHFM@SetEventNotificationMode?5for?5VM@ 0000000180005c30     libAddToBootstrapClassLoaderSearch.obj
 0002:00001c68       ??_C@_0DP@CDAABIGK@SetEventNotificationMode?5for?5NA@ 0000000180005c68     libAddToBootstrapClassLoaderSearch.obj
 0002:00001ca8       ??_C@_0DF@ODADHOND@SetEventNotificationMode?5for?5VM@ 0000000180005ca8     libAddToBootstrapClassLoaderSearch.obj
 0002:00001ce0       ??_C@_0DN@PLAPDNNM@SetEventNotificationMode?5CLASS_@ 0000000180005ce0     libAddToBootstrapClassLoaderSearch.obj
 0002:00001d20       ??_C@_09IENLFOHK@?1newclass@ 0000000180005d20     libAddToBootstrapClassLoaderSearch.obj
 0002:00001d30       ??_C@_0M@NJFOOCBM@segment?$DN?$CFs?6@ 0000000180005d30     libAddToBootstrapClassLoaderSearch.obj
 0002:00001d40       ??_C@_0CP@MODIPBOB@AddToBootStrapClassLoaderSearch@ 0000000180005d40     libAddToBootstrapClassLoaderSearch.obj
 0002:00001d70       ??_C@_0FD@OBEHNCGD@Error?3?5no?5ClassFileLoadHook?5eve@ 0000000180005d70     libAddToBootstrapClassLoaderSearch.obj
 0002:00001de0       ??_C@_1EC@JIJBPKFM@?$AAa?$AAp?$AAi?$AA?9?$AAm?$AAs?$AA?9?$AAw?$AAi?$AAn?$AA?9?$AAc?$AAo?$AAr?$AAe@ 0000000180005de0     MSVCRT:thread_safe_statics.obj
 0002:00001e28       ??_C@_1BK@MGMFAEKH@?$AAk?$AAe?$AAr?$AAn?$AAe?$AAl?$AA3?$AA2?$AA?4?$AAd?$AAl?$AAl@ 0000000180005e28     MSVCRT:thread_safe_statics.obj
 0002:00001e48       ??_C@_0BJ@JEBJOJFJ@SleepConditionVariableCS@ 0000000180005e48     MSVCRT:thread_safe_statics.obj
 0002:00001e68       ??_C@_0BJ@PGPPEPCC@WakeAllConditionVariable@ 0000000180005e68     MSVCRT:thread_safe_statics.obj
 0002:00001e88       _pDefaultRawDllMain        0000000180005e88     MSVCRT:dll_dllmain.obj
 0002:00001e88       _pRawDllMain               0000000180005e88     MSVCRT:dll_dllmain.obj
 0002:00001e90       __xmm@ffffffffffffffffffffffffffffffff 0000000180005e90     MSVCRT:utility.obj
 0002:00001ea0       _load_config_used          0000000180005ea0     MSVCRT:loadcfg.obj
 0002:00002080       _tls_used                  0000000180006080     MSVCRT:tlssup.obj
 0002:000020a8       __volatile_metadata        00000001800060a8     <linker-defined>
 0002:00002478       __rtc_iaa                  0000000180006478     MSVCRT:initsect.obj
 0002:00002480       __rtc_izz                  0000000180006480     MSVCRT:initsect.obj
 0002:00002488       __rtc_taa                  0000000180006488     MSVCRT:initsect.obj
 0002:00002490       __rtc_tzz                  0000000180006490     MSVCRT:initsect.obj
 0002:00002498       _tls_start                 0000000180006498     MSVCRT:tlssup.obj
 0002:0000249c       _Init_thread_epoch         000000018000649c     MSVCRT:thread_safe_statics.obj
 0002:000024a0       _tls_end                   00000001800064a0     MSVCRT:tlssup.obj
 0002:00002b74       __IMPORT_DESCRIPTOR_KERNEL32 0000000180006b74     kernel32:KERNEL32.dll
 0002:00002b88       __IMPORT_DESCRIPTOR_VCRUNTIME140 0000000180006b88     vcruntime:VCRUNTIME140.dll
 0002:00002b9c       __IMPORT_DESCRIPTOR_api-ms-win-crt-runtime-l1-1-0 0000000180006b9c     ucrt:api-ms-win-crt-runtime-l1-1-0.dll
 0002:00002bb0       __IMPORT_DESCRIPTOR_api-ms-win-crt-stdio-l1-1-0 0000000180006bb0     ucrt:api-ms-win-crt-stdio-l1-1-0.dll
 0002:00002bc4       __IMPORT_DESCRIPTOR_api-ms-win-crt-string-l1-1-0 0000000180006bc4     ucrt:api-ms-win-crt-string-l1-1-0.dll
 0002:00002bd8       __NULL_IMPORT_DESCRIPTOR   0000000180006bd8     kernel32:KERNEL32.dll
 0003:00000bf8       _Init_global_epoch         0000000180008bf8     MSVCRT:thread_safe_statics.obj
 0003:00000c00       __security_cookie          0000000180008c00     MSVCRT:gs_cookie.obj
 0003:00000c08       __security_cookie_complement 0000000180008c08     MSVCRT:gs_cookie.obj
 0003:00000c10       __scrt_native_dllmain_reason 0000000180008c10     MSVCRT:utility.obj
 0003:00000c18       __isa_available            0000000180008c18     MSVCRT:cpu_disp.obj
 0003:00000c1c       __isa_enabled              0000000180008c1c     MSVCRT:cpu_disp.obj
 0003:00000c20       __memset_fast_string_threshold 0000000180008c20     MSVCRT:cpu_disp.obj
 0003:00000c28       __memset_nt_threshold      0000000180008c28     MSVCRT:cpu_disp.obj
 0003:00000c30       __scrt_ucrt_dll_is_in_use  0000000180008c30     MSVCRT:ucrt_stubs.obj
 0003:00000c40       g_wrongHeapCallbacks       0000000180008c40     libAddToBootstrapClassLoaderSearch.obj
 0003:00000cc0       g_szTagInfo                0000000180008cc0     libAddToBootstrapClassLoaderSearch.obj
 0003:00002c00       g_tagFlags                 000000018000ac00     libAddToBootstrapClassLoaderSearch.obj
 0003:00002fe8       g_refsToVerifyCnt          000000018000afe8     libAddToBootstrapClassLoaderSearch.obj
 0003:00002fec       g_fakeUserData             000000018000afec     libAddToBootstrapClassLoaderSearch.obj
 0003:00002ff0       g_tagVisitCount            000000018000aff0     libAddToBootstrapClassLoaderSearch.obj
 0003:00003f90       g_refsToVerify             000000018000bf90     libAddToBootstrapClassLoaderSearch.obj
 0003:0001b690       g_userDataError            0000000180023690     libAddToBootstrapClassLoaderSearch.obj
 0003:0001b694       printdump                  0000000180023694     libAddToBootstrapClassLoaderSearch.obj
 0003:0001b988       ?_OptionsStorage@?1??__local_stdio_printf_options@@9@4_KA 0000000180023988     libAddToBootstrapClassLoaderSearch.obj
 0003:0001bf48       _tls_index                 0000000180023f48     MSVCRT:tlssup.obj
 0003:0001bf50       __scrt_current_native_startup_state 0000000180023f50     MSVCRT:utility.obj
 0003:0001bf58       __scrt_native_startup_lock 0000000180023f58     MSVCRT:utility.obj
 0003:0001bf98       __scrt_debugger_hook_flag  0000000180023f98     MSVCRT:utility_desktop.obj
 0003:0001bfa0       ?__type_info_root_node@@3U__type_info_node@@A 0000000180023fa0     MSVCRT:tncleanup.obj
 0003:0001bfb0       ?_OptionsStorage@?1??__local_stdio_scanf_options@@9@4_KA 0000000180023fb0     MSVCRT:default_local_stdio_options.obj
 0003:0001bfb8       __favor                    0000000180023fb8     MSVCRT:cpu_disp.obj
 0003:0001bfc0       __dyn_tls_init_callback    0000000180023fc0     <common>

 entry point at        0001:00002600

 Static symbols

 0000:fffda000       .debug$S                   0000000180000000     AddToBootstrapClassLoaderSearch.exp
 0000:fffda000       .debug$S                   0000000180000000     vcruntime:VCRUNTIME140.dll
 0000:fffda000       .debug$S                   0000000180000000     vcruntime:VCRUNTIME140.dll
 0000:fffda000       .debug$S                   0000000180000000     vcruntime:VCRUNTIME140.dll
 0000:fffda000       .debug$S                   0000000180000000     vcruntime:VCRUNTIME140.dll
 0000:fffda000       .debug$S                   0000000180000000     vcruntime:VCRUNTIME140.dll
 0000:fffda000       .debug$S                   0000000180000000     vcruntime:VCRUNTIME140.dll
 0000:fffda000       .debug$S                   0000000180000000     vcruntime:VCRUNTIME140.dll
 0000:fffda000       .debug$S                   0000000180000000     vcruntime:VCRUNTIME140.dll
 0000:fffda000       .debug$S                   0000000180000000     ucrt:api-ms-win-crt-convert-l1-1-0.dll
 0002:ffffc000       .idata$6                   0000000180000000     ucrt:api-ms-win-crt-convert-l1-1-0.dll
 0000:fffda000       .debug$S                   0000000180000000     ucrt:api-ms-win-crt-heap-l1-1-0.dll
 0000:fffda000       .debug$S                   0000000180000000     ucrt:api-ms-win-crt-heap-l1-1-0.dll
 0000:fffda000       .debug$S                   0000000180000000     ucrt:api-ms-win-crt-heap-l1-1-0.dll
 0000:fffda000       .debug$S                   0000000180000000     ucrt:api-ms-win-crt-heap-l1-1-0.dll
 0002:ffffc000       .idata$6                   0000000180000000     ucrt:api-ms-win-crt-heap-l1-1-0.dll
 0000:fffda000       .debug$S                   0000000180000000     ucrt:api-ms-win-crt-runtime-l1-1-0.dll
 0000:fffda000       .debug$S                   0000000180000000     ucrt:api-ms-win-crt-runtime-l1-1-0.dll
 0000:fffda000       .debug$S                   0000000180000000     ucrt:api-ms-win-crt-runtime-l1-1-0.dll
 0000:fffda000       .debug$S                   0000000180000000     ucrt:api-ms-win-crt-runtime-l1-1-0.dll
 0000:fffda000       .debug$S                   0000000180000000     ucrt:api-ms-win-crt-runtime-l1-1-0.dll
 0000:fffda000       .debug$S                   0000000180000000     ucrt:api-ms-win-crt-runtime-l1-1-0.dll
 0000:fffda000       .debug$S                   0000000180000000     ucrt:api-ms-win-crt-runtime-l1-1-0.dll
 0000:fffda000       .debug$S                   0000000180000000     ucrt:api-ms-win-crt-runtime-l1-1-0.dll
 0000:fffda000       .debug$S                   0000000180000000     ucrt:api-ms-win-crt-runtime-l1-1-0.dll
 0000:fffda000       .debug$S                   0000000180000000     ucrt:api-ms-win-crt-runtime-l1-1-0.dll
 0000:fffda000       .debug$S                   0000000180000000     ucrt:api-ms-win-crt-runtime-l1-1-0.dll
 0000:fffda000       .debug$S                   0000000180000000     ucrt:api-ms-win-crt-runtime-l1-1-0.dll
 0000:fffda000       .debug$S                   0000000180000000     ucrt:api-ms-win-crt-runtime-l1-1-0.dll
 0000:fffda000       .debug$S                   0000000180000000     ucrt:api-ms-win-crt-runtime-l1-1-0.dll
 0000:fffda000       .debug$S                   0000000180000000     ucrt:api-ms-win-crt-runtime-l1-1-0.dll
 0000:fffda000       .debug$S                   0000000180000000     ucrt:api-ms-win-crt-runtime-l1-1-0.dll
 0000:fffda000       .debug$S                   0000000180000000     ucrt:api-ms-win-crt-stdio-l1-1-0.dll
 0000:fffda000       .debug$S                   0000000180000000     ucrt:api-ms-win-crt-stdio-l1-1-0.dll
 0000:fffda000       .debug$S                   0000000180000000     ucrt:api-ms-win-crt-stdio-l1-1-0.dll
 0000:fffda000       .debug$S                   0000000180000000     ucrt:api-ms-win-crt-stdio-l1-1-0.dll
 0000:fffda000       .debug$S                   0000000180000000     ucrt:api-ms-win-crt-stdio-l1-1-0.dll
 0000:fffda000       .debug$S                   0000000180000000     ucrt:api-ms-win-crt-stdio-l1-1-0.dll
 0000:fffda000       .debug$S                   0000000180000000     ucrt:api-ms-win-crt-stdio-l1-1-0.dll
 0000:fffda000       .debug$S                   0000000180000000     ucrt:api-ms-win-crt-stdio-l1-1-0.dll
 0000:fffda000       .debug$S                   0000000180000000     ucrt:api-ms-win-crt-stdio-l1-1-0.dll
 0000:fffda000       .debug$S                   0000000180000000     ucrt:api-ms-win-crt-stdio-l1-1-0.dll
 0000:fffda000       .debug$S                   0000000180000000     ucrt:api-ms-win-crt-string-l1-1-0.dll
 0000:fffda000       .debug$S                   0000000180000000     ucrt:api-ms-win-crt-string-l1-1-0.dll
 0000:fffda000       .debug$S                   0000000180000000     ucrt:api-ms-win-crt-string-l1-1-0.dll
 0000:fffda000       .debug$S                   0000000180000000     ucrt:api-ms-win-crt-string-l1-1-0.dll
 0000:fffda000       .debug$S                   0000000180000000     ucrt:api-ms-win-crt-string-l1-1-0.dll
 0000:fffda000       .debug$S                   0000000180000000     ucrt:api-ms-win-crt-string-l1-1-0.dll
 0000:fffda000       .debug$S                   0000000180000000     ucrt:api-ms-win-crt-string-l1-1-0.dll
 0000:fffda000       .debug$S                   0000000180000000     ucrt:api-ms-win-crt-string-l1-1-0.dll
 0000:fffda000       .debug$S                   0000000180000000     kernel32:KERNEL32.dll
 0000:fffda000       .debug$S                   0000000180000000     kernel32:KERNEL32.dll
 0000:fffda000       .debug$S                   0000000180000000     kernel32:KERNEL32.dll
 0000:fffda000       .debug$S                   0000000180000000     kernel32:KERNEL32.dll
 0000:fffda000       .debug$S                   0000000180000000     kernel32:KERNEL32.dll
 0000:fffda000       .debug$S                   0000000180000000     kernel32:KERNEL32.dll
 0000:fffda000       .debug$S                   0000000180000000     kernel32:KERNEL32.dll
 0000:fffda000       .debug$S                   0000000180000000     kernel32:KERNEL32.dll
 0000:fffda000       .debug$S                   0000000180000000     kernel32:KERNEL32.dll
 0000:fffda000       .debug$S                   0000000180000000     kernel32:KERNEL32.dll
 0000:fffda000       .debug$S                   0000000180000000     kernel32:KERNEL32.dll
 0000:fffda000       .debug$S                   0000000180000000     kernel32:KERNEL32.dll
 0000:fffda000       .debug$S                   0000000180000000     kernel32:KERNEL32.dll
 0000:fffda000       .debug$S                   0000000180000000     kernel32:KERNEL32.dll
 0000:fffda000       .debug$S                   0000000180000000     kernel32:KERNEL32.dll
 0000:fffda000       .debug$S                   0000000180000000     kernel32:KERNEL32.dll
 0000:fffda000       .debug$S                   0000000180000000     kernel32:KERNEL32.dll
 0000:fffda000       .debug$S                   0000000180000000     kernel32:KERNEL32.dll
 0000:fffda000       .debug$S                   0000000180000000     kernel32:KERNEL32.dll
 0000:fffda000       .debug$S                   0000000180000000     kernel32:KERNEL32.dll
 0000:fffda000       .debug$S                   0000000180000000     kernel32:KERNEL32.dll
 0000:fffda000       .debug$S                   0000000180000000     kernel32:KERNEL32.dll
 0000:fffda000       .debug$S                   0000000180000000     kernel32:KERNEL32.dll
 0000:fffda000       .debug$S                   0000000180000000     kernel32:KERNEL32.dll
 0000:fffda000       .debug$S                   0000000180000000     kernel32:KERNEL32.dll
 0000:fffda000       .debug$S                   0000000180000000     kernel32:KERNEL32.dll
 0000:fffda000       .debug$S                   0000000180000000     kernel32:KERNEL32.dll
 0000:fffda000       .debug$S                   0000000180000000     kernel32:KERNEL32.dll
 0001:00000fe4       addRefToVerify             0000000180001fe4 f   libAddToBootstrapClassLoaderSearch.obj
 0001:00001050       agentThreadWrapper         0000000180002050 f   libAddToBootstrapClassLoaderSearch.obj
 0001:000012f4       file_basename              00000001800022f4 f   libAddToBootstrapClassLoaderSearch.obj
 0001:000019c4       startAgentThreadWrapper    00000001800029c4 f   libAddToBootstrapClassLoaderSearch.obj
 0001:00001d04       syncDebuggeeStatus         0000000180002d04 f   libAddToBootstrapClassLoaderSearch.obj
 0001:000020c4       capture_previous_context   00000001800030c4 f   MSVCRT:gs_report.obj
 0001:00002138       ?__scrt_initialize_thread_safe_statics@@YAHXZ 0000000180003138 f   MSVCRT:thread_safe_statics.obj
 0001:00002208       ?__scrt_uninitialize_thread_safe_statics@@YAXXZ 0000000180003208 f   MSVCRT:thread_safe_statics.obj
 0001:000022b0       $$000000                   00000001800032b0     MSVCRT:amdsecgs.obj
 0001:000022e0       ?dllmain_crt_dispatch@@YAHQEAUHINSTANCE__@@KQEAX@Z 00000001800032e0 f   MSVCRT:dll_dllmain.obj
 0001:00002330       ?dllmain_crt_process_attach@@YAHQEAUHINSTANCE__@@QEAX@Z 0000000180003330 f   MSVCRT:dll_dllmain.obj
 0001:00002448       ?dllmain_crt_process_detach@@YAH_N@Z 0000000180003448 f   MSVCRT:dll_dllmain.obj
 0001:000024cc       ?dllmain_dispatch@@YAHQEAUHINSTANCE__@@KQEAX@Z 00000001800034cc f   MSVCRT:dll_dllmain.obj
 0001:00002ef0       $$000000                   0000000180003ef0     MSVCRT:guard_dispatch.obj
 0001:00002f10       $$000000                   0000000180003f10     MSVCRT:guard_xfg_dispatch.obj
 0001:00002f26       ?fin$0@?0??dllmain_crt_process_attach@@YAHQEAUHINSTANCE__@@QEAX@Z@4HA 0000000180003f26 f   MSVCRT:dll_dllmain.obj
 0001:00002f3d       ?fin$0@?0??dllmain_crt_process_detach@@YAH_N@Z@4HA 0000000180003f3d f   MSVCRT:dll_dllmain.obj
 0001:00002f56       ?fin$1@?0??dllmain_crt_process_detach@@YAH_N@Z@4HA 0000000180003f56 f   MSVCRT:dll_dllmain.obj
 0001:00002f6a       ?filt$0@?0??dllmain_dispatch@@YAHQEAUHINSTANCE__@@KQEAX@Z@4HA 0000000180003f6a f   MSVCRT:dll_dllmain.obj
 0001:00002fa0       __scrt_is_nonwritable_in_current_image$filt$0 0000000180003fa0 f   MSVCRT:utility.obj
 0002:000001f8       ?__scrt_initialize_tss_var@@3P6AHXZEA 00000001800041f8     MSVCRT:thread_safe_statics.obj
 0002:00000320       ?opcLengths@@3QBEB         0000000180004320     libAddToBootstrapClassLoaderSearch.obj
 0002:00001dc8       GS_ExceptionPointers       0000000180005dc8     MSVCRT:gs_report.obj
 0002:000024a8       $unwind$fprintf            00000001800064a8     libAddToBootstrapClassLoaderSearch.obj
 0002:000024b4       $unwind$printf             00000001800064b4     libAddToBootstrapClassLoaderSearch.obj
 0002:000024c0       $unwind$?NewObject@JNIEnv_@@QEAAPEAV_jobject@@PEAV_jclass@@PEAU_jmethodID@@ZZ 00000001800064c0     libAddToBootstrapClassLoaderSearch.obj
 0002:000024c0       $unwind$nsk_lcomplain      00000001800064c0     libAddToBootstrapClassLoaderSearch.obj
 0002:000024c0       $unwind$nsk_ldisplay       00000001800064c0     libAddToBootstrapClassLoaderSearch.obj
 0002:000024c8       $unwind$nsk_lvdisplay      00000001800064c8     libAddToBootstrapClassLoaderSearch.obj
 0002:000024c8       $unwind$_RTC_Initialize    00000001800064c8     MSVCRT:initsect.obj
 0002:000024c8       $unwind$_RTC_Terminate     00000001800064c8     MSVCRT:initsect.obj
 0002:000024c8       $unwind$?__scrt_initialize_thread_safe_statics@@YAHXZ 00000001800064c8     MSVCRT:thread_safe_statics.obj
 0002:000024d4       $unwind$nsk_lvcomplain     00000001800064d4     libAddToBootstrapClassLoaderSearch.obj
 0002:000024ec       $unwind$nsk_ltrace         00000001800064ec     libAddToBootstrapClassLoaderSearch.obj
 0002:000024ec       $unwind$__report_gsfailure 00000001800064ec     MSVCRT:gs_report.obj
 0002:000024f4       $unwind$nsk_lvtrace        00000001800064f4     libAddToBootstrapClassLoaderSearch.obj
 0002:000024f4       $unwind$vmDeath            00000001800064f4     libAddToBootstrapClassLoaderSearch.obj
 0002:000024f4       $unwind$vmInit             00000001800064f4     libAddToBootstrapClassLoaderSearch.obj
 0002:000024f4       $unwind$vmStart            00000001800064f4     libAddToBootstrapClassLoaderSearch.obj
 0002:000024f4       $unwind$__raise_securityfailure 00000001800064f4     MSVCRT:gs_report.obj
 0002:000024f4       $unwind$__scrt_initialize_crt 00000001800064f4     MSVCRT:utility.obj
 0002:000024f4       $unwind$__scrt_initialize_onexit_tables 00000001800064f4     MSVCRT:utility.obj
 0002:000024f4       $unwind$__scrt_release_startup_lock 00000001800064f4     MSVCRT:utility.obj
 0002:000024f4       $unwind$__scrt_uninitialize_crt 00000001800064f4     MSVCRT:utility.obj
 0002:000024f4       $unwind$_onexit            00000001800064f4     MSVCRT:utility.obj
 0002:000024fc       $unwind$nsk_lverify        00000001800064fc     libAddToBootstrapClassLoaderSearch.obj
 0002:0000250c       $unwind$nsk_vprintf        000000018000650c     libAddToBootstrapClassLoaderSearch.obj
 0002:0000251c       $unwind$nsk_printf         000000018000651c     libAddToBootstrapClassLoaderSearch.obj
 0002:00002524       $unwind$?nsk_jni_lverify@@YAHHPEAUJNIEnv_@@HQEBDH1ZZ 0000000180006524     libAddToBootstrapClassLoaderSearch.obj
 0002:00002538       $unwind$?nsk_jni_check_exception@@YAHPEAUJNIEnv_@@QEBDH@Z 0000000180006538     libAddToBootstrapClassLoaderSearch.obj
 0002:00002554       $unwind$Java_nsk_jvmti_unit_FollowReferences_FollowRefObjects_resetTags 0000000180006554     libAddToBootstrapClassLoaderSearch.obj
 0002:00002554       $unwind$Java_nsk_jvmti_unit_functions_AddToBootstrapClassLoaderSearch_JvmtiTest_GetResult 0000000180006554     libAddToBootstrapClassLoaderSearch.obj
 0002:00002554       $unwind$addRefToVerify     0000000180006554     libAddToBootstrapClassLoaderSearch.obj
 0002:00002554       $unwind$init_callbacks     0000000180006554     libAddToBootstrapClassLoaderSearch.obj
 0002:00002554       $unwind$nsk_jvmti_resetAgentData 0000000180006554     libAddToBootstrapClassLoaderSearch.obj
 0002:00002554       $unwind$nsk_jvmti_setFailStatus 0000000180006554     libAddToBootstrapClassLoaderSearch.obj
 0002:00002554       $unwind$__scrt_initialize_default_local_stdio_options 0000000180006554     MSVCRT:default_local_stdio_options.obj
 0002:00002554       $unwind$?dllmain_crt_dispatch@@YAHQEAUHINSTANCE__@@KQEAX@Z 0000000180006554     MSVCRT:dll_dllmain.obj
 0002:00002554       $unwind$DllMain            0000000180006554     MSVCRT:dll_dllmain_stub.obj
 0002:00002554       $unwind$__GSHandlerCheck   0000000180006554     MSVCRT:gshandler.obj
 0002:00002554       $unwind$?__scrt_uninitialize_thread_safe_statics@@YAXXZ 0000000180006554     MSVCRT:thread_safe_statics.obj
 0002:00002554       $unwind$__scrt_acquire_startup_lock 0000000180006554     MSVCRT:utility.obj
 0002:00002554       $unwind$__scrt_dllmain_after_initialize_c 0000000180006554     MSVCRT:utility.obj
 0002:00002554       $unwind$__scrt_dllmain_before_initialize_c 0000000180006554     MSVCRT:utility.obj
 0002:00002554       $unwind$__scrt_dllmain_crt_thread_attach 0000000180006554     MSVCRT:utility.obj
 0002:00002554       $unwind$__scrt_dllmain_crt_thread_detach 0000000180006554     MSVCRT:utility.obj
 0002:00002554       $unwind$__scrt_dllmain_uninitialize_c 0000000180006554     MSVCRT:utility.obj
 0002:00002554       $unwind$__scrt_dllmain_uninitialize_critical 0000000180006554     MSVCRT:utility.obj
 0002:00002554       $unwind$atexit             0000000180006554     MSVCRT:utility.obj
 0002:0000255c       $unwind$nsk_jvmti_lverify  000000018000655c     libAddToBootstrapClassLoaderSearch.obj
 0002:00002570       $unwind$exitOnError        0000000180006570     libAddToBootstrapClassLoaderSearch.obj
 0002:00002580       $unwind$Java_nsk_share_jvmti_ArgumentHandler_getAgentOptionsString 0000000180006580     libAddToBootstrapClassLoaderSearch.obj
 0002:00002594       $unwind$Java_nsk_jvmti_unit_FollowReferences_FollowRefObjects_getTag 0000000180006594     libAddToBootstrapClassLoaderSearch.obj
 0002:00002594       $unwind$Java_nsk_share_jvmti_DebugeeClass_checkStatus 0000000180006594     libAddToBootstrapClassLoaderSearch.obj
 0002:00002594       $unwind$agentThreadWrapper 0000000180006594     libAddToBootstrapClassLoaderSearch.obj
 0002:000025a4       $unwind$startAgentThreadWrapper 00000001800065a4     libAddToBootstrapClassLoaderSearch.obj
 0002:000025c0       $unwind$Agent_Initialize   00000001800065c0     libAddToBootstrapClassLoaderSearch.obj
 0002:000025c0       $unwind$syncDebuggeeStatus 00000001800065c0     libAddToBootstrapClassLoaderSearch.obj
 0002:000025c0       $unwind$__scrt_dllmain_exception_filter 00000001800065c0     MSVCRT:utility.obj
 0002:000025d4       $unwind$Java_nsk_share_jvmti_DebugeeClass_resetAgentData 00000001800065d4     libAddToBootstrapClassLoaderSearch.obj
 0002:000025dc       $unwind$MA_checkStatus     00000001800065dc     libAddToBootstrapClassLoaderSearch.obj
 0002:000025f0       $unwind$Java_nsk_jvmti_unit_FollowReferences_FollowRefObjects_setTag 00000001800065f0     libAddToBootstrapClassLoaderSearch.obj
 0002:00002608       $unwind$Java_nsk_jvmti_unit_FollowReferences_FollowRefObjects_addRefToVerify 0000000180006608     libAddToBootstrapClassLoaderSearch.obj
 0002:00002624       $unwind$debug_printf       0000000180006624     libAddToBootstrapClassLoaderSearch.obj
 0002:00002630       $unwind$NativeMethodBind   0000000180006630     libAddToBootstrapClassLoaderSearch.obj
 0002:0000263c       $unwind$classFileLoadEvent 000000018000663c     libAddToBootstrapClassLoaderSearch.obj
 0002:00002644       $unwind$capture_previous_context 0000000180006644     MSVCRT:gs_report.obj
 0002:00002650       $unwind$__GSHandlerCheckCommon 0000000180006650     MSVCRT:gshandler.obj
 0002:00002658       $xdatasym                  0000000180006658     MSVCRT:amdsecgs.obj
 0002:0000265c       $unwind$?dllmain_crt_process_attach@@YAHQEAUHINSTANCE__@@QEAX@Z 000000018000665c     MSVCRT:dll_dllmain.obj
 0002:00002698       $unwind$?fin$0@?0??dllmain_crt_process_attach@@YAHQEAUHINSTANCE__@@QEAX@Z@4HA 0000000180006698     MSVCRT:dll_dllmain.obj
 0002:00002698       $unwind$?fin$0@?0??dllmain_crt_process_detach@@YAH_N@Z@4HA 0000000180006698     MSVCRT:dll_dllmain.obj
 0002:00002698       $unwind$?fin$1@?0??dllmain_crt_process_detach@@YAH_N@Z@4HA 0000000180006698     MSVCRT:dll_dllmain.obj
 0002:000026a0       $unwind$?dllmain_crt_process_detach@@YAH_N@Z 00000001800066a0     MSVCRT:dll_dllmain.obj
 0002:000026f4       $unwind$?dllmain_dispatch@@YAHQEAUHINSTANCE__@@KQEAX@Z 00000001800066f4     MSVCRT:dll_dllmain.obj
 0002:0000271c       $unwind$?filt$0@?0??dllmain_dispatch@@YAHQEAUHINSTANCE__@@KQEAX@Z@4HA 000000018000671c     MSVCRT:dll_dllmain.obj
 0002:00002724       $unwind$_DllMainCRTStartup 0000000180006724     MSVCRT:dll_dllmain.obj
 0002:00002734       $unwind$__scrt_is_nonwritable_in_current_image 0000000180006734     MSVCRT:utility.obj
 0002:00002754       $unwind$__scrt_is_nonwritable_in_current_image$filt$0 0000000180006754     MSVCRT:utility.obj
 0002:0000275c       $unwind$__scrt_fastfail    000000018000675c     MSVCRT:utility_desktop.obj
 0002:0000276c       $unwind$__security_init_cookie 000000018000676c     MSVCRT:gs_support.obj
 0002:00002778       $unwind$__isa_available_init 0000000180006778     MSVCRT:cpu_disp.obj
 0002:00002788       $xdatasym                  0000000180006788     MSVCRT:guard_dispatch.obj
 0002:00002790       $xdatasym                  0000000180006790     MSVCRT:guard_xfg_dispatch.obj
 0002:000027a0       .edata                     00000001800067a0     AddToBootstrapClassLoaderSearch.exp
 0002:000027c8       rgpv                       00000001800067c8     AddToBootstrapClassLoaderSearch.exp
 0002:00002804       rgszName                   0000000180006804     AddToBootstrapClassLoaderSearch.exp
 0002:00002840       rgwOrd                     0000000180006840     AddToBootstrapClassLoaderSearch.exp
 0002:0000285e       szName                     000000018000685e     AddToBootstrapClassLoaderSearch.exp
 0002:00002882       $N00001                    0000000180006882     AddToBootstrapClassLoaderSearch.exp
 0002:00002891       $N00002                    0000000180006891     AddToBootstrapClassLoaderSearch.exp
 0002:0000289e       $N00003                    000000018000689e     AddToBootstrapClassLoaderSearch.exp
 0002:000028e3       $N00004                    00000001800068e3     AddToBootstrapClassLoaderSearch.exp
 0002:00002920       $N00005                    0000000180006920     AddToBootstrapClassLoaderSearch.exp
 0002:00002968       $N00006                    0000000180006968     AddToBootstrapClassLoaderSearch.exp
 0002:000029a8       $N00007                    00000001800069a8     AddToBootstrapClassLoaderSearch.exp
 0002:000029e5       $N00008                    00000001800069e5     AddToBootstrapClassLoaderSearch.exp
 0002:00002a37       $N00009                    0000000180006a37     AddToBootstrapClassLoaderSearch.exp
 0002:00002a72       $N00010                    0000000180006a72     AddToBootstrapClassLoaderSearch.exp
 0002:00002aa0       $N00011                    0000000180006aa0     AddToBootstrapClassLoaderSearch.exp
 0002:00002ad1       $N00012                    0000000180006ad1     AddToBootstrapClassLoaderSearch.exp
 0002:00002b00       $N00013                    0000000180006b00     AddToBootstrapClassLoaderSearch.exp
 0002:00002b2f       $N00014                    0000000180006b2f     AddToBootstrapClassLoaderSearch.exp
 0002:00002b64       $N00015                    0000000180006b64     AddToBootstrapClassLoaderSearch.exp
 0002:00002f82       .idata$6                   0000000180006f82     kernel32:KERNEL32.dll
 0002:00002ff0       .idata$6                   0000000180006ff0     vcruntime:VCRUNTIME140.dll
 0002:00003166       .idata$6                   0000000180007166     ucrt:api-ms-win-crt-runtime-l1-1-0.dll
 0002:00003188       .idata$6                   0000000180007188     ucrt:api-ms-win-crt-stdio-l1-1-0.dll
 0002:000031a8       .idata$6                   00000001800071a8     ucrt:api-ms-win-crt-string-l1-1-0.dll
 0003:00000000       ?codeAttributeName@@3PEBDEB 0000000180008000     libAddToBootstrapClassLoaderSearch.obj
 0003:00000008       ?lineNumberAttributeName@@3PEBDEB 0000000180008008     libAddToBootstrapClassLoaderSearch.obj
 0003:00000010       ?localVarAttributeName@@3PEBDEB 0000000180008010     libAddToBootstrapClassLoaderSearch.obj
 0003:00000018       ?localVarTypeAttributeName@@3PEBDEB 0000000180008018     libAddToBootstrapClassLoaderSearch.obj
 0003:00000020       ?stackMapAttributeName@@3PEBDEB 0000000180008020     libAddToBootstrapClassLoaderSearch.obj
 0003:00000028       ?callBytes@@3PAEA          0000000180008028     libAddToBootstrapClassLoaderSearch.obj
 0003:0000002c       ?allocBytes@@3PAEA         000000018000802c     libAddToBootstrapClassLoaderSearch.obj
 0003:00000030       BOOT_CLASS                 0000000180008030     libAddToBootstrapClassLoaderSearch.obj
 0003:00000040       segment                    0000000180008040     libAddToBootstrapClassLoaderSearch.obj
 0003:0001b698       nsk_context                0000000180023698     libAddToBootstrapClassLoaderSearch.obj
 0003:0001b6a4       redefineAttempted          00000001800236a4     libAddToBootstrapClassLoaderSearch.obj
 0003:0001b6a8       redefineSucceed            00000001800236a8     libAddToBootstrapClassLoaderSearch.obj
 0003:0001b6ac       agentFailed                00000001800236ac     libAddToBootstrapClassLoaderSearch.obj
 0003:0001b6b0       context                    00000001800236b0     libAddToBootstrapClassLoaderSearch.obj
 0003:0001b768       agentThread                0000000180023768     libAddToBootstrapClassLoaderSearch.obj
 0003:0001b770       agentThreadProc            0000000180023770     libAddToBootstrapClassLoaderSearch.obj
 0003:0001b778       agentThreadArg             0000000180023778     libAddToBootstrapClassLoaderSearch.obj
 0003:0001b780       agent_data                 0000000180023780     libAddToBootstrapClassLoaderSearch.obj
 0003:0001b790       jvmti_env                  0000000180023790     libAddToBootstrapClassLoaderSearch.obj
 0003:0001b798       jvm                        0000000180023798     libAddToBootstrapClassLoaderSearch.obj
 0003:0001b7a0       jni_env                    00000001800237a0     libAddToBootstrapClassLoaderSearch.obj
 0003:0001b7a8       currentAgentStatus         00000001800237a8     libAddToBootstrapClassLoaderSearch.obj
 0003:0001b7ac       ?codeAttributeIndex@@3GA   00000001800237ac     libAddToBootstrapClassLoaderSearch.obj
 0003:0001b7b0       checkStatus_func           00000001800237b0     libAddToBootstrapClassLoaderSearch.obj
 0003:0001b7b8       ?lineNumberAttributeIndex@@3GA 00000001800237b8     libAddToBootstrapClassLoaderSearch.obj
 0003:0001b7bc       ?localVarAttributeIndex@@3GA 00000001800237bc     libAddToBootstrapClassLoaderSearch.obj
 0003:0001b7c0       ?localVarTypeAttributeIndex@@3GA 00000001800237c0     libAddToBootstrapClassLoaderSearch.obj
 0003:0001b7c4       ?stackMapAttributeIndex@@3GA 00000001800237c4     libAddToBootstrapClassLoaderSearch.obj
 0003:0001b7c8       ?stackFrameOffset@@3GA     00000001800237c8     libAddToBootstrapClassLoaderSearch.obj
 0003:0001b7cc       ?mode@@3HA                 00000001800237cc     libAddToBootstrapClassLoaderSearch.obj
 0003:0001b7d0       ?orig@@3PEBEEB             00000001800237d0     libAddToBootstrapClassLoaderSearch.obj
 0003:0001b7d8       ?gen@@3PEAEEA              00000001800237d8     libAddToBootstrapClassLoaderSearch.obj
 0003:0001b7e0       ?inputPos@@3PEAEEA         00000001800237e0     libAddToBootstrapClassLoaderSearch.obj
 0003:0001b7e8       ?endPos@@3PEBEEB           00000001800237e8     libAddToBootstrapClassLoaderSearch.obj
 0003:0001b7f0       ?genPos@@3PEAEEA           00000001800237f0     libAddToBootstrapClassLoaderSearch.obj
 0003:0001b7f8       ?markPos@@3PEAEEA          00000001800237f8     libAddToBootstrapClassLoaderSearch.obj
 0003:0001b800       ?constantPool@@3PEAPEADEA  0000000180023800     libAddToBootstrapClassLoaderSearch.obj
 0003:0001b808       ?constantPoolSize@@3GA     0000000180023808     libAddToBootstrapClassLoaderSearch.obj
 0003:0001b80c       ?constantPoolCount@@3GA    000000018002380c     libAddToBootstrapClassLoaderSearch.obj
 0003:0001b810       ?zeroBytes@@3PAEA          0000000180023810     libAddToBootstrapClassLoaderSearch.obj
 0003:0001b814       ?codeLength@@3IA           0000000180023814     libAddToBootstrapClassLoaderSearch.obj
 0003:0001b818       ?map@@3PEAIEA              0000000180023818     libAddToBootstrapClassLoaderSearch.obj
 0003:0001b820       ?widening@@3PEACEA         0000000180023820     libAddToBootstrapClassLoaderSearch.obj
 0003:0001b828       jvmti                      0000000180023828     libAddToBootstrapClassLoaderSearch.obj
 0003:0001b830       iGlobalStatus              0000000180023830     libAddToBootstrapClassLoaderSearch.obj
 0003:0001b834       boot_class_count           0000000180023834     libAddToBootstrapClassLoaderSearch.obj
 0003:0001b838       jvmti_caps                 0000000180023838     libAddToBootstrapClassLoaderSearch.obj
 0003:0001b850       callbacks                  0000000180023850     libAddToBootstrapClassLoaderSearch.obj
 0003:0001b990       GS_ExceptionRecord         0000000180023990     MSVCRT:gs_report.obj
 0003:0001ba30       GS_ContextRecord           0000000180023a30     MSVCRT:gs_report.obj
 0003:0001bf00       ?g_tss_cv@@3U_RTL_CONDITION_VARIABLE@@A 0000000180023f00     MSVCRT:thread_safe_statics.obj
 0003:0001bf08       ?g_tss_event@@3PEAXEA      0000000180023f08     MSVCRT:thread_safe_statics.obj
 0003:0001bf10       ?g_tss_mutex@@3U_RTL_CRITICAL_SECTION@@A 0000000180023f10     MSVCRT:thread_safe_statics.obj
 0003:0001bf38       ?g_sleep_condition_variable_cs@@3P6AHPEAU_RTL_CONDITION_VARIABLE@@PEAU_RTL_CRITICAL_SECTION@@K@ZEA 0000000180023f38     MSVCRT:thread_safe_statics.obj
 0003:0001bf40       ?g_wake_all_condition_variable@@3P6AXPEAU_RTL_CONDITION_VARIABLE@@@ZEA 0000000180023f40     MSVCRT:thread_safe_statics.obj
 0003:0001bf4c       ?__proc_attached@@3HA      0000000180023f4c     MSVCRT:dll_dllmain.obj
 0003:0001bf60       ?is_initialized_as_dll@@3_NA 0000000180023f60     MSVCRT:utility.obj
 0003:0001bf61       ?module_local_atexit_table_initialized@@3_NA 0000000180023f61     MSVCRT:utility.obj
 0003:0001bf68       ?module_local_atexit_table@@3U_onexit_table_t@@A 0000000180023f68     MSVCRT:utility.obj
 0003:0001bf80       ?module_local_at_quick_exit_table@@3U_onexit_table_t@@A 0000000180023f80     MSVCRT:utility.obj
